:020000040800F2
:10700000A017002099710008997F0008897E000868
:10701000957F0008457A0008798900080000000083
:1070200000000000000000000000000031840008A3
:10703000557C000800000000AF710008B171000825
:10704000B3710008B3710008B37100089982000899
:10705000B3710008B3710008B3710008B371000880
:10706000B3710008B3710008B3710008B371000870
:10707000B3710008B3710008B3710008B371000860
:10708000B3710008B3710008B3710008B371000850
:10709000B3710008B3710008B3710008B371000840
:1070A000B3710008B3710008B3710008B371000830
:1070B000B3710008A5850008B3710008B37100081A
:1070C000B3710008B3710008B3710008B371000810
:1070D000B371000875870008B3710008B371000828
:1070E000B3710008B3710008B371000800F002F832
:1070F00000F042F80AA090E8000C82448344AAF110
:107100000107DA4501D100F037F8AFF2090EBAE80D
:107110000F0013F0010F18BFFB1A43F001031847CB
:10712000987F0000B87F0000103A24BF78C878C16B
:10713000FAD8520724BF30C830C144BF04680C607D
:10714000704700000023002400250026103A28BFC5
:1071500078C1FBD8520728BF30C148BF0B607047C9
:10716000642900F09D80732900F09B820020704705
:107170001FB51FBD10B510BD00F0D2FA1146FFF7C4
:10718000F7FF03F03DFD00F0F0FA03B4FFF7F2FF64
:1071900003BC00F0F5FA00000948804709480047A1
:1071A000FEE7FEE7FEE7FEE7FEE7FEE7FEE7FEE7B7
:1071B000FEE7FEE704480549054A064B7047000014
:1071C00045850008ED700008A0050020A0170020EC
:1071D000A0070020A00700200FB41CB5074B06AA8B
:1071E0007B4469460090059800F031FA002069461A
:1071F00000F040FA1CBC5DF814FB00009104000094
:1072000070B5044685690068C10601D5302600E0E6
:107210002026C00707D070BDD4E901213046904731
:10722000206A401C20626D1EF6D570BD70B5044604
:1072300085690078C00707D170BDD4E901212020FD
:107240009047206A401C20626D1EF6D570BD70B557
:107250000C460546012A05D02878800600D5EA6943
:10726000002302E0012305E05B1C934202D2E05CB4
:107270000028F9D1A869E618C01AA861286A18443C
:1072800028622846FFF7BCFF04E0D5E9012114F885
:10729000010B9047B442F8D32846FFF7C7FF70BDF3
:1072A0002DE9F0410646002410687529314616A5DF
:1072B00010D0AFF30080002802DA404213A507E0A7
:1072C00031688A0701D512A502E0490704D511A546
:1072D000012401E0AFF3008000210A2206F1240717
:1072E00009E0B0FBF2FCB0FBF2F302FB1C00303013
:1072F00078541846491C0028F3D123462A463046C4
:10730000BDE8F04100F044B9000000002D0000008D
:107310002B000000200000002DE9F0474FF0000A8C
:1073200089460446C0F820A02046E1688847002826
:1073300076D0252806D0D4E901219047206A401C48
:107340002062F1E7E168204600258847C4F81CA0C8
:1073500006460027C4F818A02A2E09D0304601F0AE
:1073600074FB38B304EB8708303EC8F8186019E0A6
:1073700059F8041B204604EB87029161E1688847B5
:10738000012F064618D1E069002820DA25F02005F3
:107390001DE0D8F8180000EB800006EB4000303804
:1073A000C8F818002046E1688847064601F04DFB02
:1073B0000028EED1012F0AD02E2E08D12046E168F8
:1073C00088477F1C0646022F45F02005C4DBA069D4
:1073D000002803DA404245F00105A061E80701D02A
:1073E00025F01005B6B1A6F14100192802D82036C3
:1073F00045F400654A463146204625604D46FFF774
:10740000AFFE58B1012806D0ED1D25F0070000F1B0
:10741000080989E704E005F1040985E730468AE7B1
:10742000206ABDE8F08730B505460B462A4613F8BA
:10743000014B12F8010B08B1A042F8D01CB1002892
:1074400002D06D1CF1E7284630BD40EA010310B5BB
:107450009B070FD1042A0DD310C808C9121F9C42E4
:10746000F8D020BA19BA884201D9012010BD4FF0D6
:10747000FF3010BD1AB1D30703D0521C07E0002023
:1074800010BD10F8013B11F8014B1B1B07D110F880
:10749000013B11F8014B1B1B01D1921EF1D1184683
:1074A00010BD40EA0103024630B59B0710D14FF0F2
:1074B000013400E008C208C91D1B9D4315EAC41F22
:1074C000F8D013F0FF0102F8011B0DD01B0AF8E7FA
:1074D00011F8013B002B02F8013B05D011F8013BEC
:1074E000002B02F8013BF3D130BD032A40F230807B
:1074F00010F0030C00F0158011F8013BBCF1020FF5
:10750000624498BF11F801CB00F8013B38BF11F875
:10751000013BA2F1040298BF00F801CB38BF00F88C
:10752000013B11F0030300F0C080083AC0F008806E
:1075300051F8043B083A51F804CBA0E80810F5E7ED
:10754000121D5CBF51F8043B40F8043BAFF30080D0
:10755000D20724BF11F8013B11F801CB48BF11F845
:10756000012B24BF00F8013B00F801CB48BF00F815
:10757000012B704770477047704710B500F0C8F88E
:10758000006810BD10B5044600F0C2F8046010BDDC
:107590002DE9F0470D4699469246044600F124082D
:1075A0000168880604D5E06921F01001216000E03F
:1075B0000120A84201DD471B00E00027A1697A19DC
:1075C00002EB0900081AA0612078C00602D4204608
:1075D000FFF716FE002608E0D4E901211AF806009C
:1075E0009047206A401C761C20624E45F4DB2078D0
:1075F000C0060AD52046FFF703FE06E0D4E90121C4
:1076000030209047206A401C2062381EA7F10107F5
:10761000F4DC07E0D4E9012118F805009047206A5E
:10762000401C2062281EA5F10105F3DC2046FFF76F
:10763000FDFD2078000602D50220BDE8F08701207C
:10764000FBE7000001694A1C02610878704700B539
:107650008FB0CDE901310021059105497944CDE98B
:10766000031011466846FFF757FE0FB000BD00003B
:10767000E5FFFFFF0A6802F8010B0A60704710B5CA
:10768000436913B1AFF3008001E0FFF7E0FD012093
:1076900010BD127800F124010A7000224A70012204
:1076A000EDE711684FF0FF32E9E710B5203AC0F07E
:1076B0000B80B1E81850203AA0E81850B1E81850F3
:1076C000A0E81850BFF4F5AF5FEA027C24BFB1E830
:1076D0001850A0E8185044BF18C918C0BDE81040A1
:1076E0005FEA827C24BF51F8043B40F8043B08BFAA
:1076F0007047D20728BF31F8023B48BF11F8012B71
:1077000028BF20F8023B48BF00F8012B704700005B
:1077100000487047400500200048704740050020A1
:107720007546FFF7F9FFAE4605006946534620F05F
:107730000700854618B020B5FFF73CFDBDE82040A6
:107740004FF000064FF000074FF000084FF0000B1D
:1077500021F00701AC46ACE8C009ACE8C009ACE8D0
:10776000C009ACE8C0098D46704710B50446AFF3B8
:1077700000802046BDE81040FFF707BD70470000BD
:1077800001491820ABBEFEE72600020000B585B017
:107790004FF4004000F050FC1E4800F053F8002069
:1077A000009001208DF804008DF805004FF4602052
:1077B00002900020039002208DF8100069461548C1
:1077C00000F082F8072301220221124800F0A4F8F9
:1077D0000723022205210F4800F09EF801210D48E1
:1077E00000F025F801210B4800F016F8094800F0D8
:1077F000EFF800BF074800F05DF80028FAD105480F
:1078000000F0F6F800BF034800F04AF80028FAD16B
:1078100005B000BD0024014021B1826842F00102A0
:10782000826003E0826822F001028260704721B129
:10783000826842F48072826003E0826822F480727F
:107840008260704710B504461248844208D1012175
:10785000401500F02DFC0021601500F029FC17E018
:107860000D48844208D10121001500F021FC0021BF
:10787000201500F01DFC0BE00848844208D10121CE
:10788000C80300F015FC00214FF4004000F010FC8C
:1078900010BD00000024014000280140003C0140D0
:1078A000014600208A6802F004020AB1012000E0CB
:1078B00000207047014600208A6802F008020AB1E1
:1078C000012000E00020704730B502460020002370
:1078D00050680F4C20400D790C6844EA0524204381
:1078E000506090680B4C2040D1E902542C434D79F4
:1078F00044EA450420439060D06A20F470000C7C78
:10790000641EE4B2234340EA0350D06230BD00005D
:10791000FFFEF0FFFDF7F1FFF0B504460D46002035
:107920000021092D11DDE068A5F10A0606EB4607E6
:10793000072606FA07F18843A5F10A0606EB460674
:1079400003FA06F10843E0600CE0206905EB450707
:10795000072606FA07F1884305EB450603FA06F108
:1079600008432061072A0FDA606B561E06EB860774
:107970001F2606FA07F18843561E06EB860605FA0F
:1079800006F10843606322E00D2A0FDA206BD61F50
:1079900006EB86071F2606FA07F18843D61F06EB7B
:1079A000860605FA06F10843206310E0E06AA2F1BA
:1079B0000D0606EB86071F2606FA07F18843A2F19B
:1079C0000D0606EB860605FA06F10843E062F0BDF7
:1079D000816841F008018160704721B1826842F4FA
:1079E000A002826003E0826822F4A00282607047F5
:1079F000816841F004018160704710B5012000F0FA
:107A000067FB002000F064FB10BD000008B50146D4
:107A100000200090034800900098084400900098CF
:107A2000008808BD006C004008B500220092044A9E
:107A30000092009A02440092009A116008BD000072
:107A4000006C004000BFFEE7014601EBC1000522CB
:107A500090FBF2F000F5A07080B2704721B102688F
:107A600042F00102026004E002684FF6FE731A4021
:107A70000260704700B58BB00121084600F0E8FABB
:107A80000F4800F023F80F4800900F4801900020A5
:107A90000290142003900020049080200590400064
:107AA0000690800007902020089000020990002096
:107AB0000A906946024800F0AFF80BB000BD000024
:107AC000080002404C2401406804002001684FF681
:107AD000FE72114001600021016041608160C1605F
:107AE0004B49884208D14A490839496841F00F0199
:107AF000474A083A51608AE045491431884208D122
:107B000043490839496841F0F001414A083A516057
:107B10007DE03F492831884208D13D49083949680C
:107B200041F470613A4A083A516070E038493C319A
:107B3000884208D136490839496841F47041344ACD
:107B4000083A516063E032495031884208D13049E7
:107B50000839496841F470212D4A083A516056E0CD
:107B60002B496431884208D129490839496841F4D0
:107B70007001274A083A516049E025497831884226
:107B800008D123490839496841F07061204A083A10
:107B900051603CE01F49884206D1011F096841F04D
:107BA0000F01021F116032E01A491431884208D1D6
:107BB0001849091F096841F0F001164A121F1160A7
:107BC00025E014492831884208D11249091F096863
:107BD00041F470610F4A121F116018E00D493C31E9
:107BE000884208D10B49091F096841F47041094ACC
:107BF000121F11600BE007495031884207D1054937
:107C0000091F096841F47021024A121F1160704770
:107C1000080002400804024010B50022026847F63E
:107C2000F0739A430C6A8B6823430C6923434C69B5
:107C300023438C692343CC6923434C6A23438C6AD6
:107C400023431A430260CB6843600B6883604B6830
:107C5000C36010BD70470146A1F5A07202EB82021D
:107C600090B2092290FBF2F290B270472DE9F041F8
:107C7000024600250026002000230024002791F85A
:107C800003C00CF00F0591F803C00CF0100CBCF110
:107C9000000F03D091F802C04CEA050591F800C02E
:107CA000BCF1000F31D0146800202BE04FF0010C24
:107CB0000CFA00F3B1F800C00CEA03069E4220D192
:107CC00083004FF00F0C0CFA03F7BC4305FA03FCDA
:107CD0004CEA040491F803C0BCF1280F06D14FF020
:107CE000010C0CFA00FCC2F814C00AE091F803C0C1
:107CF000BCF1480F05D14FF0010C0CFA00FCC2F8A2
:107D000010C0401C0828D1D31460B1F800C0BCF1E9
:107D1000FF0F34DD546800202EE000F1080C4FF016
:107D2000010808FA0CF3B1F800C00CEA03069E4201
:107D300021D183004FF00F0C0CFA03F7BC4305FA76
:107D400003FC4CEA040491F803C0BCF1280F05D1F0
:107D500000F1080C08FA0CF8C2F8148091F803C07E
:107D6000BCF1480F07D100F1080C4FF0010808FAE8
:107D70000CF8C2F81080401C0828CED35460BDE82F
:107D8000F0810000F0B50A46002300240021002500
:107D900000F00046B6F1004F02D11D4EF16901E03E
:107DA0001B4E7168C0F3034583B200F44016B6F56C
:107DB000401F08D121F07061154E766826F070667C
:107DC000134F7E6012E000F48016B6F5801F06D1D6
:107DD000032606FA05F4A14341F0706106E0460D62
:107DE000360103FA06F6B14341F0706122B1460D47
:107DF000360103FA06F6314300F00046B6F1004FB3
:107E000002D1034EF16101E0014E7160F0BD00004E
:107E1000000001400246002093680B400BB1012096
:107E200000E0002070470146C86880B270470246F3
:107E30000020D3680B400BB1012000E00020704708
:107E40004161704701617047C160704770B502467B
:107E50000D46FF21FF23002409E012F8010B80EA00
:107E600001040748005D80EA03010648035D281EFF
:107E7000A5F10106B5B2F0D143EA012070BD0000C2
:107E80006AEE00086AEF000800BFFEE710B502F0D6
:107E9000BFFB4FF480710F48FFF7D4FF40210E481D
:107EA000FFF7D0FF02210C48FFF7CCFF4FF4007121
:107EB0000848FFF7C5FF4FF47A7001F041F94FF41D
:107EC00000710448FFF7BEFF4FF4FA7001F038F973
:107ED00010BD0000000C01400008014070B50446D0
:107EE0004FF400511148FFF7ABFF02F0E9FA1048D8
:107EF000FFF799FF00F47F4040EA040529460C484B
:107F0000FFF7A2FF4FF480710948FFF799FF0221A4
:107F10000848FFF795FF02210648FFF793FF4FF44B
:107F200080710348FFF78EFF70BD00000010014014
:107F3000000C01400008014070B504464FF40051A8
:107F40001148FFF77FFF02F0BBFA1048FFF76BFF05
:107F500000F47F4040EA040529460C48FFF774FF0F
:107F60004FF480710948FFF76BFF02210848FFF7C3
:107F700067FF02210648FFF765FF4FF48071034851
:107F8000FFF760FF70BD000000100140000C0140D1
:107F90000008014000BFFEE7704710B54FF4A06035
:107FA00000F03AF810BD000070B5002100230F2248
:107FB000C47804B3154C246804F4E064C4F5E064A8
:107FC000210AC1F10403CA40447804FA03F1847819
:107FD0001440214309010E4C0678A155047804F0A1
:107FE0001F050124AC4005786D11AD0005F1E025B9
:107FF000C5F8004109E0047804F01F050124AC40F5
:10800000044D0678761145F8264070BD0CED00E071
:1080100000E400E080E100E002490143024A11600F
:10802000704700000000FA050CED00E0014908620D
:108030007047000000000E4201460020034A5068CD
:1080400020F4404008435060704700000010024098
:1080500029B1064A52690243044B5A6104E0034ABB
:1080600052698243014B5A61704700000010024080
:1080700029B1064AD2690243044BDA6104E0034A9B
:10808000D2698243014BDA61704700000010024060
:1080900029B1064A92690243044B9A6104E0034AFB
:1080A00092698243014B9A617047000000100240C0
:1080B00029B1064AD2680243044BDA6004E0034A5D
:1080C000D2688243014BDA60704700000010024022
:1080D00001490860704700004004424230B5002169
:1080E0000022002400232D4D6D6805F00C0121B104
:1080F000042905D0082923D105E0294D056022E097
:10810000274D05601FE0254D6D6805F47012234D65
:108110006D6805F48034022505EB92421CB9214DAF
:10812000554305600BE01D4D6D6805F400351DB12C
:108130001C4D5543056002E0194D5543056002E0B2
:10814000174D056000BF00BF144D6D6805F0F001CC
:108150000909154D6B5C0568DD4045600F4D6D6884
:1081600005F4E061090A104D6B5C4568DD408560EF
:108170000A4D6D6805F46051C90A0B4D6B5C45688A
:10818000DD40C560054D6D6805F44041890B074D24
:108190006B5CC568B5FBF3F5056130BD00100240AE
:1081A00000127A0000093D000A0000201A00002099
:1081B00010B501460022002300204A11012A02D1F5
:1081C000094C236806E0022A02D1074C236A01E029
:1081D000054C636A01F01F02012494401C400CB15D
:1081E000012000E0002010BD0010024000210B4AD9
:1081F00011700A4A203A82F82010012802D004287F
:1082000008D103E00121054A117004E00521034A69
:10821000117000E000BF00BF704700002010024056
:1082200001490860704700003C0442420249096A63
:108230000143014A11627047001002400249098857
:108240008143014A11807047042800400348008898
:1082500040F01000014908807047000004280040E9
:10826000034800884FF6EF710840014908807047C5
:108270000428004001460020064A12880A40D0B275
:10828000044A121F12880A4012B108B1012000E00E
:10829000002070470428004010B50120FFF7EAFFD6
:1082A000002866D002F008FF38480068010C0C2056
:1082B000FFF7BAFB3548008881B21020FFF7B4FB06
:1082C000334801881420FFF7AFFB4FF400613148B9
:1082D000FFF7ADFD20B101211820FFF7A5FB03E05A
:1082E00000211820FFF7A0FB2948008820B128486A
:1082F0000088401E264908802748007820B126487B
:108300000078401E244908702448007820B1234892
:108310000078401E214908702148007820B120488B
:108320000078401E1E4908701E48007820B11D4884
:108330000078401E1B4908701B48008828B11A4865
:108340000088401E1849088013E01848C07A0128A8
:108350000FD181020F48FFF76AFD50B11448007831
:1083600038B91448007820B94FF480610948FFF704
:1083700067FD0220FFF77EFF10B10220FFF75EFFCE
:108380000520FFF75BFF00F037F810BD7C000020F0
:1083900072000020000C0140840000203300002007
:1083A0006C0000208500002082000020FA040020DC
:1083B0006F0000207000002029B1064A1288024395
:1083C000044B1A8004E0034A12888243014B1A804E
:1083D000704700000028004000B50246FFF736FF56
:1083E000C2F3034003490880091D0A80FFF738FFE4
:1083F00000BD00000828004000BF0348008800F0CE
:1084000020000028F9D07047042800400748008861
:108410004FF6F77108400549088000BF03480088FF
:1084200000F008000028F9D0704700000428004040
:10843000704710B500F002F810BD00000CB5002028
:10844000019000903348006840F480303149086062
:1084500000BF3048006800F4003000900198401CD4
:108460000190009820B94FF6FF7101988842F0D131
:108470002848006800F4003010B10120009001E0AD
:10848000002000900098012843D12348006840F064
:108490001000214908600846006820F003000860C9
:1084A0000846006840F0020008601A484068194910
:1084B00048600846406848600846406840F480606C
:1084C00048600846406820F47C10486008464068D0
:1084D00040F4F81048600846006840F0807008607A
:1084E00000BF0C48006800F000700028F9D009486F
:1084F000406820F00300074948600846406840F0A3
:108500000200486000BF0348406800F00C000828E3
:10851000F9D10CBD0010024000200240042808D10F
:108520004FF0E021096941F004014FF0E0221161B0
:1085300007E04FF0E021096921F004014FF0E0224B
:108540001161704710B51248006840F001001049F1
:108550000860084640680F4908400D4948600846D1
:1085600000680D4908400A4908600846006820F480
:10857000802008600846406820F4FE0048604FF400
:108580001F008860FFF755FF04480549086010BDCB
:10859000001002400000FFF8FFFFF6FE0070000828
:1085A00008ED00E010B50121164800F076F808B398
:1085B0000121144800F062F80120134908701348A3
:1085C00000780A2805DA11480078401C0F49087025
:1085D00017E002F039FE00200C49087001200C4918
:1085E00008700C480078322805DA0A480078401CE8
:1085F0000849087005E00020064908700120064976
:10860000087010BD0004004022000020250000205A
:108610002300002026000020240000207FB505460E
:108620000C4601210220FFF723FDADF80850ADF8FC
:1086300004400020ADF80A00ADF8060001A90E487C
:1086400000F046F8012211460B4800F037F81D20D3
:108650008DF8000001208DF8010003208DF8020044
:1086600001208DF803006846FFF79EFC01210248B7
:1086700000F007F87FBD000000040040CA430282FA
:10868000704721B1028842F00102028004E00288B2
:108690004FF6FE731A400280704730B50246002044
:1086A00000230024158A05EA0103958905EA0104DF
:1086B00013B10CB1012000E0002030BD1AB1838954
:1086C0000B43838102E083898B43838170470000E1
:1086D000002202881D4B98420ED01D4B98420BD0B1
:1086E000B0F1804F08D01B4B984205D01A4B9842EE
:1086F00002D01A4B984204D14FF68F731A404B8820
:108700001A43174B984207D0164B984204D04FF6A5
:10871000FF431A40CB881A4302808B8883850B88DD
:1087200003850A4B98420BD0094B984208D00E4B58
:10873000984205D00D4B984202D00D4B984201D182
:108740000B7A03860123838270470000002C0140CE
:10875000003401400004004000080040000C0040CC
:10876000001000400014004000400140004401405F
:108770000048014010B520211F4800F05EF8012894
:1087800015D11E480078C82802DB00201B4908705C
:108790001949091D0988CAB218490878411C174BA4
:1087A000197017490A5400201649087023E0402127
:1087B000114800F042F801281DD140210E4800F078
:1087C00027F80E4800781049097888420ADA0B49E0
:1087D0000878411C094A11700949095C064A121DB2
:1087E000118008E080210948FFF72AFB0020034997
:1087F00008700549087010BD0038014028000020AD
:10880000A0030020270000202900002000080140CC
:1088100001F40072B2F5007F00D100BFCA430280AC
:10882000704721B1828942F40052828104E082893A
:108830004DF6FF731A408281704702460020B1F561
:10884000007F00D100BF13880B400BB1012000E076
:1088500000207047F0B503460024002600250020C4
:1088600040F66A17B94200D100BF1846C1F342145E
:1088700001F01F06012707FA06F5012C01D10C3083
:1088800004E0022C01D1103000E014301AB1076866
:108890002F43076002E00768AF430760F0BD0000A8
:1088A0002DE9F04786B005460E460024A24600BFDB
:1088B000A1460027B08900B100BF2F462C8A4CF694
:1088C000FF700440F08804432C82AC894EF6F3100C
:1088D0000440B08831890843718908430443AC815E
:1088E000AC8A4FF6FF400440B0890443AC8201A833
:1088F000FFF7F4FB1F48874202D1DDF810A001E02A
:10890000DDF80CA0A88900F4004040B10AEBCA00D1
:1089100000EB0A1031684900B0FBF1F807E00AEB00
:10892000CA0000EB0A1031688900B0FBF1F864203E
:10893000B8FBF0F004012009642101FB1089A8892B
:1089400000F4004040B1322000EBC900B0FBF1F070
:1089500000F00700044308E0322000EB0910642116
:10896000B0FBF1F000F00F0004432C8106B0BDE82D
:10897000F08700000038014000BFFEE72DE9F0411C
:108980004F1E00EBC7010446D1E9000115461E4603
:1089900037F006020DD02A46334603F0A9FB7F1EAE
:1089A00004EBC703D3E9002303F0F8F837F006021D
:1089B000F1D1022F25D0042F13D0062F18BFBDE808
:1089C000F0812A46334603F093FBD4E90A2303F0EF
:1089D000E5F82A46334603F08BFBD4E9082303F07D
:1089E000DDF82A46334603F083FBD4E9062303F07F
:1089F000D5F82A46334603F07BFBD4E9042303F081
:108A0000CDF82A46334603F073FBD4E9022303F082
:108A1000C5F82A46334603F06BFBD4E90023BDE8D2
:108A2000F04103F0BBB80000002213461046014994
:108A300003F070B90000F03F012203F07FBD002277
:108A400013461046114603F065B930380A2801D2A2
:108A5000012070470020704710B50022002014E06C
:108A6000002107E00A4B03EB810333F810301A446E
:108A70004B1CD9B20A29F5DB0A23B2FBF3F3054CF0
:108A800024F810300022431CD8B20228E8DB10BDC5
:108A9000680400202A00002008B501214802FFF7E1
:108AA000F7FA48208DF803000420ADF8000069466D
:108AB0000C48FFF7DBF800208DF803002020ADF80C
:108AC000000069460748FFF7D1F8FEF75FFEFEF7A2
:108AD000D1FF01210448FEF780FF01210348FEF782
:108AE000BDFF08BD0008014000240140080002400D
:108AF0002DE9F0410446002500264FF6FF77AC46ED
:108B00000FE0208805443AB12088B04200DD268875
:108B10002088B84200DA2788A41C0CF101001FFA53
:108B200080FC8C45EDDBF01BC82802DD01201870AD
:108B300001E00020187042B1A81BA0EB0708881EB6
:108B4000B8FBF0F080B2BDE8F081B5FBF1F080B287
:108B5000F9E700002DE9F04F8BB056480078132854
:108B600005DA54480078401C5249087002E00020A1
:108B70005049087001F0B0F94F494E4A127821F877
:108B800012000AAB012214214B48FFF7B1FF8246C5
:108B90004FF4FA500AFB00F0CAF58051B0FBF1FB2C
:108BA000584603F091FACDE9000101F07BFECDE9D2
:108BB00002010020414901F075FE8046DDE90223F3
:108BC00003F0A0FB00223E4BCDE9040103F090FA34
:108BD00000223C4BCDE9060103F088FB06463246F5
:108BE0000B460020384903F095F804460022374B25
:108BF00003F088FBCDE9080103F020FA00B2344904
:108C000008800846B0F9000010F1C80F08DB0846DC
:108C1000B0F90000B0F5487F02DC9DF8280018B1DB
:108C200001202C49087002E000202A4908702849D8
:108C3000098888B2FEF708FF00B2274908800120A2
:108C4000244908700846007830BB24480078022880
:108C50000AD12348007838B91F480078214909789B
:108C6000401A40B2204908701C48007830B11B48B7
:108C7000007802280BD11A48007840B116480088C5
:108C8000194991F90010401A1849088008E0154860
:108C900000881649088003E01248008813490880BC
:108CA00012480088FEF7D7FF114908800BB0BDE8D5
:108CB000F08F000057000020900400200088C3407F
:108CC00000A0724000DCAE408F7366410054A540A6
:108CD0005000002055000020520000205E000020BF
:108CE0005600002066000020540000206400002090
:108CF000620000202DE9F04385B004460B34A778CC
:108D0000E07840EA07272579607940EA05250B3CA1
:108D10000C22B2492046FEF798FB002878D10B348C
:108D20006078102875D1C82FFCD14FF000084FF0A3
:108D300002090020AA490880AA48C07A012817D150
:108D4000C102A948FFF773F8F8B1A848007838B114
:108D5000A348008820F00100401CA149088022E0BF
:108D60009F48008820F00200801C9D4908801AE07E
:108D70004FF400619C48FFF75AF838B198480088D2
:108D800020F00100401C964908800CE04FF48061FF
:108D90009548FFF74CF830B19148008820F0020068
:108DA000801C8F4908804FF480719148FFF73FF88D
:108DB00020B908218E48FFF73AF830B1884800887A
:108DC00020F00400001D8649088010218848FFF724
:108DD0002EF830B18248008820F008000830804921
:108DE00008808048C17A7E48008861F305107C497C
:108DF00008807E48007810B97E48007850B17848E5
:108E0000008820F4004000F500407549088007E024
:108E10009CE0D1E07248008820F40040704908804E
:108E2000754800887549097808446D49098860F3D8
:108E30008E116B48018000880012ADF80000684870
:108E40000088ADF80200072D04D04FF003084FF062
:108E5000010969E0E579207A40EA0525684805803E
:108E60004FF6FF70854206D15E48407A18B901205E
:108E70006449087002E0002062490870657AA07AAF
:108E800040EA052557484580E57A207B40EA0525DC
:108E900054488580657BA07B40EA052551498D714A
:108EA000E57B207C40EA05250D72657CA07C40EACC
:108EB0000525CD71E57C207D40EA05254D724FF0FA
:108EC00002090846407A02280FD140F28A204C4914
:108ED0000880444880790988A1EB4000401E414940
:108EE000488008464088888012E03E48407A03283F
:108EF0000ED140F28A20424908803A488079098898
:108F000001EB4000401C3749488008464088888073
:108F100034494888FEF79FFE3B49088031498888DC
:108F2000FEF799FE394908800B3C43464A4669469C
:108F3000204601F045FF0546284602F099F800203A
:108F40003349087002203349087044E0002606E0E7
:108F5000A05D10B105B0BDE8F083701CC6B20C2E48
:108F6000F6DB0B346078042835D1642F33D1012D22
:108F700031D12948007800B32648007801281CD157
:108F800026480078C8B10020234908708046072091
:108F9000ADF800000B3C1148016821604168616038
:108FA0008068A060434601226946204601F008FF20
:108FB0000546284602F05CF80DE01648007818B91E
:108FC00001201449087006E012480078012802D1F7
:108FD00000200F49087000BFBCE700001E050020FC
:108FE00088000020FA040020000C01406F000020DF
:108FF0000008014070000020720000208500002061
:109000006600002056000020680000206A00002052
:109010005F0000205E00002030000020760000206D
:1090200010B590B01348006801901248001D006808
:1090300002901048083000680390002409E00E49AF
:1090400001EB4400B0F8E80F0AA921F81400601CF5
:10905000C4B20C2CF3DB04A901A800F00FF818220D
:1090600004A90AA8FEF7F1F910B9012010B010BD4B
:109070000020FBE7E8F7FF1F0060000818B500229A
:10908000009211E002780B4B9DF800401A5510F841
:10909000012B01F8012B9DF8002001F8012B9DF810
:1090A0000020521CD2B200929DF800200C2AE9DB6D
:1090B00018BD00001E05002010B504466FF0040026
:1090C000FFF72CFAE11704EB5171C1F3C701074A0E
:1090D00011701046007800EB4001C1EBC0104FF654
:1090E000FF7101EAC0000249088010BD1E00002087
:1090F000200000200146114A12884A434FF0E02325
:109100005A6100229A611A46126942F001021A61FC
:1091100000BF4FF0E022106900F001021AB100F424
:109120008032002AF5D04FF0E022126922F00102CD
:109130004FF0E0231A6100229A617047200000205E
:1091400000BF411E88B20028FBD170470146114A7A
:1091500012784A434FF0E0235A6100229A611A467E
:10916000126942F001021A6100BF4FF0E02210695B
:1091700000F001021AB100F48032002AF5D04FF05D
:10918000E022126922F001024FF0E0231A6100226E
:109190009A6170471E00002010B500F029F80120E8
:1091A00001F0D0F901242246641C0B48007804FB2E
:1091B0000020C1B209A2272001F050FB2246641C06
:1091C0000548007804FB0020C1B205A2032001F08D
:1091D00045FB02F06DFC10BD090000204D43550019
:1091E000446576696365204944204572726F720058
:1091F00000200021084A00BF0BE0002004E000230B
:1092000002F8013B431CD8B26028F8DB01F10803E7
:10921000D9B24029F1DB7047A000002010B5FFF75C
:10922000E7FF022001F08EF917A20421084601F0A1
:1092300015FB18A21421042001F010FB052001F0F9
:1092400081F91748C089B8B11548C0893C2190FB05
:10925000F1F4224613A11448FDF7BEFF124A28215B
:10926000084601F0FBFA022001F06CF90FA2302150
:109270003A2001F0F3FA04E00DA22821082001F0C1
:10928000EDFA02F015FC10BD20486F742053746194
:109290007274000020202044656C61790000000099
:1092A000FA040020256400002A0500206D696E0084
:1092B000204F4646000000007CB5FFF799FF0520CF
:1092C00001F040F9EE480078022803D0ED4800781C
:1092D00000286ED1EA48007801286AD0EA48408820
:1092E0000028FAD0E848407A012805D1E7A21421E5
:1092F000182001F0B3FAB4E1E348407A022803D021
:10930000E148407A032805D1E1A21421202001F090
:10931000A5FAECE0DC48C07900287CD0DA48007A75
:1093200010B1D948448801E0D74884880A20B4FBAA
:10933000F0F63246D7A1D848FDF74EFFB4F57A7F54
:1093400005D3D54A0821182001F088FA04E0D24A52
:109350000821242001F082FAD04800884FF6FF71DE
:10936000884204D1CEA1CC48FDF736FF09E0CB48B6
:1093700000880A2190FBF1F63246C6A1C648FDF7E7
:109380002BFFC6480088B0F57A7F05DBC24A222150
:10939000182001F063FA04E0BF4A2221242001F0E2
:1093A0005DFA012001F0CEF8B4F57A7F02D30425EE
:1093B00001E038E1002505F14401C8B2B9A210214D
:1093C00001F04CFA0120009005F14201CAB2491E99
:1093D0000190C8B21123102102F03CFBAF48008875
:1093E000B0F57A7F01DB042500E0002505F144019A
:1093F000C8B2ACA22A2101F031FA0120009005F197
:109400004201CAB2491E0190C8B22B232A2102F0A0
:1094100021FB62E0FFE79C48007A10B1A248048873
:1094200001E0A24804880A20B4FBF0F6324699A174
:109430009948FDF7D1FEB4F57A7F05D3964A082105
:10944000182001F00BFA04E0934A0821242001F0CF
:1094500005FA924800884FF6FF71884204D190A126
:109460008D48FDF7B9FE09E0914800880A2190FB7C
:10947000F1F6324687A18848FDF7AEFE874800889E
:10948000B0F57A7F05DB844A2221182001F0E6F945
:1094900004E0814A2221242001F0E0F9012001F0BA
:1094A00051F884A21021442001F0D8F90120009045
:1094B0001123422210210190412002F0CBFA7DA21B
:1094C0002A21442001F0CAF9012000902B234222D6
:1094D0002A210190412002F0BDFA77A200211C2030
:1094E00001F0BCF977A23821202001F0B7F9012062
:1094F00001F028F863480078D0B96148007830B1AD
:109500005F480078022813D17048007880B1704815
:10951000007848B16F4A0021522000F073FF6EA21C
:109520000A215A2001F09AF901206C49087002E0E2
:1095300000206A4908706A48007848B35248C07AE7
:1095400001280AD1C1026748FEF771FC28B96648B4
:10955000008810B15E48007878B94FF40061614826
:10956000FEF765FC48B94848C07A012810D04FF48E
:1095700080615C48FEF75BFC50B15CA218210020C2
:1095800001F06CF95BA22221062001F067F921E0CD
:1095900059480078F0B14FF400615248FEF747FC9B
:1095A00040B95148008810B95448007810B1484873
:1095B000007828B94FF400614A48FEF738FC48B1FA
:1095C0004FA21821002001F049F94AA222210620C9
:1095D00001F044F92C48807A90B146A21C21542015
:1095E00001F03CF92848407A90BB01200321212357
:1095F0004C22CDE900101F211A2002F02BFA30E096
:1096000041A21C21482001F029F91F48407AF8B9ED
:109610000120032121234422CDE900101F211A201B
:1096200002F018FA1DE01648007890B1022000F010
:1096300089FF37A20021084601F010F938A2142151
:10964000002001F00BF939A22821042001F006F9CD
:1096500007E0022000F076FF36A21821042001F076
:10966000FDF83748007838B1012000F06BFF35A2D3
:109670000021084601F0F2F802F01AFA7CBD000061
:109680005E00002055000020FA0400204F464600EE
:109690004F4E0000253264002A050020640000209F
:1096A0002D2D2D0046000000680000206A000020DB
:1096B0006200002043000000536574706F696E748F
:1096C0000000000043757272656E74005600002041
:1096D0006E00002058EE00083200000074000020E8
:1096E00070000020000C0140720000204865617489
:1096F000000000004F6E00006F0000207500002089
:10970000436F6F6C000000004175746F0000000033
:10971000506C6561736520707265737300000000A2
:109720002041646472657373696E67002020202095
:109730004B65790020204F66666C696E65000000FD
:109740004F00002065657072000000001CB5FFF737
:109750004FFD022000F0F6FE15A20421002001F0CA
:109760007DF816A21421002001F078F81648427BFB
:1097700016A11748FDF730FD1348407B0A2805DB8A
:10978000134A2A21242001F069F804E0104A2A2112
:10979000282001F063F8022003213A233C22CDE97E
:1097A00000102821222002F055F902F081F91CBD99
:1097B00020436F6D70726573736F72002064656C07
:1097C00061792074696D6500FA04002025647300D6
:1097D0002A05002010B5FFF70BFD022000F0B2FEB5
:1097E0000AA20A21002001F039F8012000F0AAFEA7
:1097F0000AA22321042001F031F80CA23221042016
:1098000001F02CF802F054F910BD000052657365A8
:10981000742053797374656D000000004144445214
:1098200020746F20636F6E6669726D002020464160
:109830004E20746F206261636B00000010B5FFF76B
:10984000D7FC022000F07EFE0AA20821002001F0D1
:1098500005F80CA21C21002001F000F8012000F006
:1098600071FE0BA23221002000F0F8FF02F020F977
:1098700010BD000052657365742053797374656D73
:109880000000000020202020446F6E6500000000D2
:1098900020506C6561736520526573746172740049
:1098A00010B5FFF7A5FC4348C07A00281FD102205D
:1098B00000F048FE40A20521042000F0CFFF012067
:1098C00000F040FE3FA21921032000F0C7FF41A293
:1098D0002321002000F0C2FF43A22D21002000F030
:1098E000BDFF46A23721032000F0B8FF5FE03148FA
:1098F000C07A03281AD1022000F024FE43A20521D9
:10990000042000F0ABFF012000F01CFE42A2192150
:10991000032000F0A3FF44A22321002000F09EFFBB
:1099200045A22D21002000F099FF40E02148C07A97
:10993000022819D100F006FE42A20521042000F001
:109940008DFF012000F0FEFD41A21921002000F052
:1099500085FF43A22321032000F080FF36A22D21A2
:10996000002000F07BFF22E01248C07A01281ED1BF
:10997000022000F0E7FD3EA20521042000F06EFF6A
:10998000012000F0DFFD0FA21921032000F066FF87
:109990003AA22321002000F061FF13A22D21002014
:1099A00000F05CFF39A23721032000F057FF02F0DE
:1099B0007FF810BDFA04002020486561742F436FC2
:1099C0006F6C000057697468206F72207769746843
:1099D0006F7574004D756C7469706C65207374617B
:1099E0006765732E0000000041646A75737420621D
:1099F0007920776972696E67000000002020205787
:109A00002C57322C592C59320000000020436F6F24
:109A10006C206F6E6C790000202043656E7472615B
:109A20006C206169720000002020636F6E646974AD
:109A3000696F6E696E6700002020202020206F6E05
:109A40006C7900002048656174206F6E6C790000AD
:109A50002020204761732C6F696C206F720000001A
:109A600020656C65637472696320686561740000C9
:109A700020486561742070756D70000020617578F4
:109A8000696C69617279206865617400202020200A
:109A9000204155582F45000010B5FFF7A9FB1E487F
:109AA000007B00281AD0022000F04CFD1BA20A21E6
:109AB000042000F0D3FE012000F044FD1AA21E2174
:109AC000002000F0CBFE1CA22821002000F0C6FEE2
:109AD0001EA23221002000F0C1FE19E0022000F099
:109AE00031FD1FA20A21042000F0B8FE012000F081
:109AF00029FD0DA21E21002000F0B0FE1BA228218E
:109B0000002000F0ABFE11A23221002000F0A6FEE2
:109B100001F0CEFF10BD0000FA0400202020436FAA
:109B20006F6C696E670000002041207769726520C4
:109B30006C6162656C656400224F2220636F6E6EFB
:109B4000656374656420746F0000000074686520AC
:109B50004F2F42207465726D696E616C00000000C9
:109B6000202048656174696E67000000224222204F
:109B7000636F6E6E656374656420746F000000002F
:109B800010B5FFF735FB022000F0DCFC084A0A2183
:109B9000202000F063FE074A07A10948FDF71CFBDF
:109BA000074A1E21042000F059FE01F081FF10BD7C
:109BB000EA040020E0040020202020562025730025
:109BC0002A05002008B501210420FEF761FA0320D0
:109BD0008DF8020010208DF80300C001ADF80000E0
:109BE00069460848FEF742F84FF48050ADF800008F
:109BF00014208DF8030069460248FEF737F800F09C
:109C0000B2F908BD000801402DE9F04707460C46AF
:109C100090461D46DDF8209000260AE000F010FA7C
:109C2000384600F0D1F900B905E000F014FA701CD4
:109C3000C6B2C82EF2DB00BFC82E02DB0120BDE891
:109C4000F087B8F1020F09D1C4F3072000F0BCF986
:109C5000012803D100F0FFF90120F0E7E0B200F0A5
:109C6000B3F9012803D100F0F6F90120E7E700F08D
:109C7000E7F947F0010000F0A7F9B8B90BE000F0F0
:109C80007BF905F8010BB9F1000F02D000F05AF989
:109C900001E000F049F9B9F10000A9F1010101F07A
:109CA000FF09ECD100F0D7F90020C8E700F0D3F9A4
:109CB0000120C4E72DE9F04782460C461746984636
:109CC000DDE9089541E000260AE000F0B9F95046C8
:109CD00000F07AF900B905E000F0BDF9701CC6B2D9
:109CE000C82EF2DB00BFC82E02DB0120BDE8F087E2
:109CF000022F09D1C4F3072000F066F9012803D12F
:109D000000F0A9F90120F1E7E0B200F05DF90128C7
:109D100003D100F0A0F90120E8E711E019F8010BE8
:109D200000F052F9012803D100F095F90120DDE798
:109D3000681EC5B2641CA8F10100204000B901E012
:109D4000002DEBD100BF00F086F9002DBBD1002023
:109D5000CCE7000010B525480078002844D000204A
:109D60002249087022480078012802D101F000FD44
:109D700001E001F057FC4FF400411E48FEF757F890
:109D8000F0B91D480078022808D01B480078B8B9FF
:109D90001A480078A0B11A48408888B1194800884C
:109DA000401C80B21749088041F27071884207DB7D
:109DB0000020144908804FF400410E48FEF742F895
:109DC0000D480078012808D00B48007850B90B489E
:109DD000007810B10A48408820B94FF40041054886
:109DE000FEF72EF8FEF7B6FE10BD0000230000209F
:109DF00076000020000801405E0000207400002072
:109E0000FA0400205C00002010B50548007830B14D
:109E100000200349087001F00BF9FEF71DFE10BD8C
:109E20002200002010B52248007800283FD00020F2
:109E30001F4908701F48007858B11F480078401C1F
:109E4000C0B21D4908700A2803DB002008701949B8
:109E500008701A48007858B119480078401CC0B200
:109E600017490870022803DB0020087013490870A6
:109E700000F0F8FF00F06CF91048007840B111488C
:109E8000007828B10F480078401E0E49087002E0A3
:109E900000200A4908700C48007818B100200A49CF
:109EA000087004E008480078401C0749087010BD9D
:109EB000240000205E0000205F0000203000002011
:109EC00060000020320000206E0000200148408821
:109ED000704700006804002002480088C0F30B00AF
:109EE000704700002A00002008B501210C20FEF771
:109EF000CFF803208DF8020010208DF803004FF4F6
:109F00008C70ADF8000069460548FDF7AFFE4FF4D0
:109F10004060ADF8000069460248FDF7A7FE08BDA5
:109F200000080140000C014010B5002001F07CFA4F
:109F3000012001F08BFA012001F076FA002001F0F7
:109F400073FA10BD10B5002001F06EFA002001F088
:109F50007DFA012001F068FA002001F065FA012085
:109F600001F074FA10BD10B5012001F06FFA012064
:109F700001F05AFA10BD000070B5012529031148FF
:109F8000FDF760FF00BF002001F04EFA6006040EEE
:109F90000A20FFF7DBF8012001F046FA4FF4805168
:109FA0000848FDF737FF08B144F001046806050EC4
:109FB000002DE8D1002001F037FA0A20FFF7C6F89B
:109FC000204670BD0008014070B50546802400BFE2
:109FD000002001F029FA05EA040001F037FA0A200E
:109FE000FFF7B4F8012001F01FFA0A20FFF7AEF8DE
:109FF0006410002CECD1002001F016FA4FF48051CF
:10A000000E48FDF71FFF0A20FFF7A0F8012001F01E
:10A010000BFA0A20FFF79AF84FF480510748FDF732
:10A02000F9FE0646002001F0FFF90A20FFF78EF83E
:10A030000EB1012070BD0020FCE7000000080140C7
:10A0400010B5012001F002FA012001F0EDF9002025
:10A0500001F0FCF910BD10B5002001F0E5F9002079
:10A0600001F0F4F9012001F0DFF9012001F0EEF92F
:10A0700010BD704710B52048007803280ED11F4846
:10A08000007B18B100201D49087302E001201B4924
:10A09000087301F031FDFFF7FFFC2BE01648007854
:10A0A000042811D11548407B002805DD1348407B6A
:10A0B000401E1249487302E014201049487301F011
:10A0C0001BFDFFF743FB15E00B480078052811D175
:10A0D0000A48C0893C2805DB0848C0893C38074944
:10A0E000C88103E04FF496700449C88101F004FD73
:10A0F000FFF794F810BD000076000020FA0400205D
:10A1000010B510480078E0B90F48C07A012818D17E
:10A110000E480078012808D103200C49087005205A
:10A1200008490870FFF7B8FC0BE0084800780328DE
:10A1300007D1012005490870052002490870FFF782
:10A14000BBF810BD33000020FA0400207600002088
:10A1500010B515480078012815D11448007830B1A1
:10A1600003280BD0042806D005280AD100E009E016
:10A1700000F0E4F806E0FFF7C3FF03E000F05CF84E
:10A1800000E000BF00BF0A48007858B109480078D5
:10A19000401CC0B207490870052803DB0020087086
:10A1A0000349087010BD000031000020410000206C
:10A1B000450000204600002010B51A48007801280C
:10A1C00005D11949087002201849087023E0154884
:10A1D000007806280AD1072012490870012000F0F3
:10A1E00013FF01F011F8FFF729FB14E00D48007888
:10A1F000052810D10E48C089F02805DC0C48C0891C
:10A200003C300B49C88102E000200949C881FFF7B2
:10A2100005F801F071FC07480078401C05490870FA
:10A2200010BD000076000020300000203200002029
:10A23000FA0400204500002010B512480078F8B953
:10A240001148007801280BD110480078022807D166
:10A2500005200D4908700B490870FEF7DFFF0FE07D
:10A2600009480078042803D007480078052807D15A
:10A27000012005490870052002490870FFF71CF805
:10A2800010BD000033000020760000205E0000209A
:10A2900010B52848007802281FD12748C07A30B16D
:10A2A000012808D002280AD0032810D10BE0012091
:10A2B0002149C8720BE002201F49C87207E0032041
:10A2C0001D49C87203E000201B49C87200BF00BFCF
:10A2D00001F012FCFFF7E4FA2AE01648007804289F
:10A2E00011D11548407B142805DA1348407B401CE7
:10A2F0001149487302E000200F49487301F0FCFB4C
:10A30000FFF724FA14E00B480078052810D10A481A
:10A31000C089F02805DC0848C0893C300649C8815E
:10A3200002E000200449C88101F0E6FBFEF776FF59
:10A3300010BD000076000020FA04002010B50E4881
:10A340000078C0B90D480078012808D102200B49D7
:10A350000870052008490870FFF7A2FA0BE00748CB
:10A360000078022807D1012004490870052002491D
:10A370000870FEF7A1FF10BD33000020760000201A
:10A3800010B51B480078062803D101201849087031
:10A390002DE018480078032808DB002015490870D4
:10A3A000062013490870FFF715FA20E012480078DC
:10A3B00040B911480078D0B910480078B8B11048B9
:10A3C0004088A0B10E48407A88B909480078012831
:10A3D0000DD10B48807A18B100200949887202E03B
:10A3E00001200749887201F087FBFEF765FF10BD69
:10A3F00076000020450000205E0000207400002050
:10A40000FA0400202DE9F84F80468946154615F8D4
:10A4100001AB15F8010B00900AF00707082F15D2C1
:10A42000DFE807F00406080A0C0E101280240EE084
:10A4300001240CE002240AE0042408E0082406E0D9
:10A44000102404E0202402E0402400E000BF00BF0C
:10A450004FF0000B2AE0B9F1400F00DD2DE0274658
:10A4600000261CE008EB0600602800DD19E02878D3
:10A47000384038B108EB0601C8B20122494601F064
:10A480006BFB06E008EB0601C8B20022494601F06A
:10A4900063FB7F100FB980276D1C701CC6B2564538
:10A4A000E0DB00BF09F1010000F0FF095846411C44
:10A4B00001F0FF0B00998842CDDB00BFBDE8F88FAB
:10A4C00008B501210820FDF7E3FDFF20ADF80000ED
:10A4D00003208DF8020010208DF80300694609481A
:10A4E000FDF7C4FB01210846FDF7D2FD0121064816
:10A4F000FDF748FC1820ADF8000069460148FDF75B
:10A50000B5FB08BD000C0140000230002DE9F0470A
:10A5100006460F4690469946DDF820A034460CE0EA
:10A520003D4606E052462946204601F015FB681CD0
:10A53000C5B24D45F6DD601CC4B24445F0DDBDE852
:10A54000F0870000014606294DD2DFE801F04C03F8
:10A5500012212E3D0822254B1A700622244B1A7018
:10A560000822244B1A705001234A121A234B1A60F6
:10A570003AE010221D4B1A7008221D4B1A7010224F
:10A580001C4B1A7050011E4A121A1C4B1A602BE009
:10A590000822164B1A70164B1A70164B1A7050017F
:10A5A000184A121A154B1A601EE00C220F4B1A7033
:10A5B00008220F4B1A700C220E4B1A705001124ACF
:10A5C000121A0E4B1A600FE03022084B1A7010223C
:10A5D000074B1A701822074B1A7090010B4A121A77
:10A5E000064B1A6000E000BF00BF7047000000206B
:10A5F0000800002009000020C8C500080400002051
:10A6000058D20008C0C80008D8CD000888DC00086F
:10A6100008B501211C20FDF73BFD4220ADF80000EC
:10A6200010208DF8030003208DF8020069461E48B3
:10A63000FDF71CFB40F2FF30ADF8000010208DF854
:10A64000030003208DF8020069461848FDF70EFB51
:10A650004FF40050ADF8000010208DF803000320E7
:10A660008DF8020069461248FDF700FB01210846FB
:10A67000FDF70EFD01210F48FDF784FB4FF400406C
:10A68000ADF8000003208DF8020010208DF80300C3
:10A6900069460548FDF7EAFA1820ADF8000069465A
:10A6A0000248FDF7E3FA08BD00080140000C014034
:10A6B00000100140000230002DE9F04F04460D4625
:10A6C0009046994600274FF0010B4D4507DD66B2D5
:10A6D000444606F0FF086EB24D4606F0FF09A8EBAF
:10A6E000040046B2A9EB05004FFA80FA294620463D
:10A6F000099A01F031FA002E04DCA4EB080046B2FE
:10A700004FF0FF3B56451CDD18E0002F06DD681CAE
:10A71000C5B2AAEB0600384447B202E007EB0A00D4
:10A7200047B204EB0B00C4B2602C01DA402D00DB11
:10A7300006E029462046099A01F00EFA4445E4D184
:10A740001BE017E0002F07DD04EB0B00C4B2A6EB03
:10A750000A00384447B201E0B81947B2681CC5B2D4
:10A76000602C01DA402D00DB06E029462046099ADC
:10A7700001F0F2F94D45E5D100BFBDE8F08F0000D2
:10A780002DE9F04706460F469246304800683049AA
:10A7900009780AFB0109002551E099F8008000249E
:10A7A00044E0072C16DC08F0800038B17A19D1B2E9
:10A7B0003219D0B2012201F0CFF906E07A19D1B2F4
:10A7C0003219D0B2002201F0C7F94FEA48604FEACF
:10A7D000106826E009F10100814690F80080082405
:10A7E0001AE008F0800038B17A19D1B23219D0B22B
:10A7F000012201F0B1F906E07A19D1B23219D0B2D2
:10A80000002201F0A9F94FEA48604FEA1068602C75
:10A8100000DD05E0601CC4B20E4800788442E0DB35
:10A8200000BF602C00DD05E0601CC4B20948007860
:10A830008442B6DB00BF09F10109681CC5B20648B5
:10A8400000788542A9DBBDE8F08700000400002005
:10A8500000000020080000200900002070B5054617
:10A860000E46144615E00D4800782844602800DDA7
:10A8700012E00B4800783044402800DD0CE02278DC
:10A8800031462846FFF77CFF044800782844C5B2CB
:10A89000641C20780028E6D100BF70BD08000020AD
:10A8A000090000202DE9F04DC84A002490B09142E3
:10A8B00005DA21F00043934201D805D120B110B050
:10A8C000BDE8F04DFEF7B8B8B1F5801F1BDA53EACA
:10A8D000000209D0002911DA0120FCF753FE10B064
:10A8E000BDE8F04DFEF7ABB80220FCF74BFEFEF7DB
:10A8F0009BF810B081F00041BDE8F08D6FF0350499
:10A90000362201F01BFE04EB2152C1F31308B049BB
:10A91000A2F2FF33414401F4801282F07F6103EB25
:10A92000225281F04051009241EA08010022A94BD5
:10A9300001F0E8FC044608F10200A74EC0F3130042
:10A940000D467E44032867D2D6E90023204601F055
:10A9500039FB1ED10098002802BFD6E9000110B0D3
:10A96000BDE8F08D01F099FB07460C469B4A9C4BD5
:10A9700001F0BEFB06460D469A4A9B4B38462146DF
:10A9800001F0B6FB10B032462B46BDE8F04D01F0A9
:10A9900005B94FF05532954B2046294601F0A8FBEA
:10A9A0000022934B01F0A2FC06460F4622462B469E
:10A9B0001046194601F09CFB32463B4601F098FBDD
:10A9C000064600980F46F0B101F067FB80468A46C4
:10A9D000824A834B01F08CFB32463B4601F086FCF9
:10A9E00022462B4601F08EFC05460C467D4A7E4BE6
:10A9F0004046514601F07CFB10B02A462346BDE894
:10AA0000F04D01F07FBC0B4610B03246204629467F
:10AA1000BDE8F04D01F076BC00224FF080432046A7
:10AA200001F0BCF802460B462046294601F072F9B7
:10AA300006460F46009801F030FBCDE9040132468E
:10AA40003B461046394601F053FB0C9069480C9A7E
:10AA50004044019009910B46104601F049FB8246A3
:10AA6000024665488B46C8F151080B4608F5D728C1
:10AA700003217844FDF782FF52465B4601F038FB24
:10AA80000A905E480D9152465B4604217844FDF7DA
:10AA900075FF099B0C9A01F02BFB844601980D9BD6
:10AAA00040EA080860460A9A01F078F8834608915F
:10AAB000B8F1000F4EDD4FF0FF322046294601F07D
:10AAC0003DFD22462B4601F013FB804600988A4646
:10AAD00060B3DDE90401414A414B01F009FB0991F2
:10AAE00000905A4640465146089B01F057F83246BE
:10AAF0003B4601F0FDFA099B009A01F04FF84246EF
:10AB0000534601F0F3FB22462B4601F0FBFB0446C3
:10AB10000D46DDE90401334A334B01F0E9FA10B088
:10AB200022462B46BDE8F04D01F0ECBB5A464046AC
:10AB3000089B01F033F832463B4601F0D9FA424611
:10AB4000534601F0D3FB10B022462B46BDE8F04D32
:10AB500001F0CCBB009840B3DDE904011F4A204B53
:10AB600001F0C6FA80468A465A4620462946089B86
:10AB700001F0C8FB32463B4601F0BAFA4246534662
:10AB800001F0C0FB22462B4601F0BCFB04460D46FB
:10AB9000DDE90401134A144B01F0AAFA10B0224671
:10ABA0002B46BDE8F04D01F0ADBB0B465A462046A2
:10ABB000294601F0A7FB32463B4601F099FA10B056
:10ABC00022462B46BDE8F04D01F090BB0000F07F1F
:10ABD000645F09000000F03F6A470000763C793569
:10ABE000EF39EA3D0000E0FE422EE63F5555D53FE5
:10ABF0000000E03F86EBF9FF02460000004600003F
:10AC00005E4800685E49B0FBF1F0C5B22846FEF729
:10AC100053FAFDF7C2F901214FF0C050FDF728FAB1
:10AC20000120FDF703FAFEF7CDFF544800685549AF
:10AC3000B0FBF1F0401E85B229466320FDF7EEFC23
:10AC400000F02EFDFDF728FFFFF74EF9FDF71EF986
:10AC5000E220FDF743F9E020FDF740F9A320FDF7DE
:10AC60003DF9A020FDF73AF9C820FDF737F9AC20EF
:10AC7000FDF734F9A620FDF731F9A420FDF72EF9F0
:10AC80002C20FDF72BF92E20FDF728F92F20FDF7BA
:10AC900025F92520FDF722F98120FDF71FF908206D
:10ACA000FDF71CF9D520FDF719F90020FDF716F97D
:10ACB000D220FDF713F90020FDF710F94020FDF731
:10ACC0000DF9B020FDF70AF91020FDF707F9002073
:10ACD000FDF704F94FF49670FEF70CFAAF20FDF77C
:10ACE000FDF84FF400412848FDF7AAF8FEF798F95F
:10ACF00018B9FEF751FA00BFFEE724492448FCF7D3
:10AD0000D0FB24A12248FCF78EFB044634B1211D60
:10AD10002148FCF7C6FB641E00202070FEF730FFC0
:10AD200000201E4908701E49088000F0F7F800F066
:10AD3000D7F94FF400611B48FDF782F84FF48061AA
:10AD40001848FDF77DF810210F48FDF779F800202D
:10AD5000154908701549087015494880154908704B
:10AD60003C201549087000201449087005E0FFF7E1
:10AD70004BF8FEF7EFFFFFF755F8F8E78C000020DF
:10AD800040420F00A0860100000801406AF0000860
:10AD9000EA04002056455200E0040020760000201E
:10ADA00078000020000C01406F000020700000209F
:10ADB000FA04002054000020860000206D000020CE
:10ADC0002DE9F04704460F4690469946B9F1000F29
:10ADD00007D0207B40F08001217384F80D900E2570
:10ADE00030E0207B04281AD10D254FEA4860020E7E
:10ADF00029466D1C625400260EE037F81600021238
:10AE00002846691CCDB2225417F816202846691C22
:10AE1000CDB22254701CC6B24645EEDB12E0207B58
:10AE2000052802D0207B10280CD10D25002607E034
:10AE300017F816202846691CCDB22254701CC6B2E1
:10AE40004645F5DB29462046FDF700F882464FEAE5
:10AE50002A206055611981F801A0A81CC0B2BDE884
:10AE6000F087000010B51848007868B917480088C6
:10AE7000401C80B215490880042823DB002008808C
:10AE80000120114908701DE00F480078012808D101
:10AE90000F48007810B9FEF70FFA13E0FFF758F9E2
:10AEA00010E00A480088401C80B2084908807828D1
:10AEB00008DB0020088004480078072802D0012021
:10AEC0000149087010BD00007600002078000020C5
:10AED0003100002070B505460C4620780F281ADD99
:10AEE0002078284410F8026C2078284410F8010CCF
:10AEF00040EA06262078801E81B22846FCF7A6FF8D
:10AF0000B04205D1002020702846FDF7F3FE04E092
:10AF10000020207001E00020207070BD38B51224A0
:10AF200000BF402CFDDC1C4B01220021AE20009410
:10AF3000FEF76AFE012802D11849087002E00020DD
:10AF400016490870A01E81B21348FCF77FFF124912
:10AF5000098A88421AD0104B01224021AE20009469
:10AF6000FEF752FE012802D10C49087002E00020D1
:10AF70000A490870A01E81B20748FCF767FF06491E
:10AF8000098A884202D0012000F03EF82246024998
:10AF90000348FCF7AAFA38BDFA0400204F0000204D
:10AFA0000C05002010B5FEF791FF044640F63C70FA
:10AFB000844203DD00201349087021E040F6485028
:10AFC000844203DD01200F49087019E040F68C200F
:10AFD000844203DD02200B49087011E040F26C70DE
:10AFE000844203DD03200749087009E0B4F5AF7F10
:10AFF00003DD04200349087002E0052001490870C0
:10B0000010BD00003900002010B50446002007499B
:10B0100088720320C87201200873002048734FF41F
:10B020009670C88100F068FD10BD0000FA04002091
:10B0300010B580210A48FCF7FAFE80B9094800786B
:10B04000401CC0B207490870022808DB00200870C5
:10B050000548007818B104490448FFF73BFF10BDCC
:10B06000000801402700002028000020A003002045
:10B0700010B5044600200A4908700A48047080216F
:10B080000948FCF7DFFE0020084908700878411CD9
:10B09000064A11700649095C064A118010BD00007D
:10B0A000270000202900002000080140280000207F
:10B0B000A0030020043801400748008807490860C1
:10B0C00008460088000408600348001D00880968DD
:10B0D0000844024908607047182800407C0000209E
:10B0E00070B500260420FCF791FC012832D0012124
:10B0F0004FF0C050FCF7BCFF0120FCF797FFFCF7B6
:10B100007CFC0120FDF772F800BF4120FDF750F8EC
:10B110000028FAD04FF48070FDF788F80120FDF781
:10B120007FF8FDF769F9FDF771F901210846FDF790
:10B1300043F9FDF761F9FDF789F847F6FF70FDF770
:10B140004BF9FDF759F9FDF78BF801210420FCF7C5
:10B150006BFC07E0FDF75AF901210846FDF72CF9D1
:10B16000FDF74AF9FFF7A8FF0C20FCF74FFC064655
:10B170001020FCF74BFC40EA06461420FCF746FC86
:10B1800004461820FCF742FC054604B9F5B135B178
:10B190001248C08912490968891B441A03E0104803
:10B1A0000068801B241A002C03DA00200D49088057
:10B1B00001E00C490C800948C0890A490988884285
:10B1C00007DA0648C0890749088002E000200549DF
:10B1D000088000F009F8002070BD0000FA0400208B
:10B1E0007C0000207200002008B503208DF80000CC
:10B1F00000208DF801008DF8020001208DF8030079
:10B200006846FCF7D1FE08BD10B501214FF0C050D3
:10B21000FCF72EFF0120FCF709FFFCF7EEFB0021F5
:10B220000120FDF7C9F8FDF7E7F80020FCF7F8FF6B
:10B230000020FCF7DBFF0020FCF7F8FE00214FF0B8
:10B24000C050FCF715FF10BD10B5FFF7ABFE60480E
:10B250000078062879D2DFE800F0034E5C6A79872F
:10B260005C480078002845D15B48007818B9002078
:10B270005A4908703EE05A48006800283AD05848B9
:10B28000006805282FD956480068B0F5967F2AD265
:10B2900051480078514908700846007818B30846AC
:10B2A0000078062813D2DFE800F0120C0903060F1D
:10B2B000FEF782FF0CE0FEF7DDFE09E0FFF760F825
:10B2C00006E0FEF7D6FE03E0FEF7E2FF00E000BF77
:10B2D00000BF4FF400414348FCF7B2FD0020424953
:10B2E0000880424908800020414908703C490860B4
:10B2F0004049087047E037480078012808D13648AF
:10B300000078012804D136480068401C34490860A0
:10B3100039E030480078022808D12F480078022808
:10B3200004D12F480068401C2D4908602BE02948B3
:10B330000078032808D128480078032804D1284839
:10B340000068401C264908601DE01BE02148007889
:10B35000042808D120480078042804D12048006837
:10B36000401C1F4908600EE01A480078052808D1E3
:10B3700019480078052804D119480068401C18496C
:10B38000086000E000BF00BF124800781249087052
:10B390000F4800780F49087011480068B0F5967F93
:10B3A00015D90F480068401E0D490860012010495A
:10B3B000087007480078104908704FF400410948A8
:10B3C000FCF73EFD0020084908800849088010BDB0
:10B3D0003900002037000020380000204000002005
:10B3E0003C000020000801405C00002078000020A4
:10B3F000310000203600002041000020064800787F
:10B4000048B10020044908700448C08904490880F4
:10B410003C2004490880704780000020FA04002086
:10B42000720000208200002010B504462CB14FF4B9
:10B4300000610548FCF706FD04E04FF40061024896
:10B44000FCF7FEFC10BD00000008014010B50446EA
:10B450002CB14FF480510548FCF7F4FC04E04FF4A4
:10B4600080510248FCF7ECFC10BD000000080140D0
:10B4700010B52D48008800284ED12C48C07A0128EC
:10B480001FD12A48007B70B14FF480612848FCF737
:10B49000CEFCB0B90320274908704FF480612448DE
:10B4A000FCF7D0FC0DE04FF480612148FCF7BFFCB5
:10B4B00038B103201F4908704FF480611C48FCF725
:10B4C000BFFC1C48007838BB4FF400611848FCF7FB
:10B4D000AEFC80B918480078184908701848007800
:10B4E00048B91848007830B91048407B14490870B2
:10B4F0000120144908701248007850B911480078AA
:10B50000012806D1C1020A48FCF79CFC00200D4925
:10B51000087001200C49087001200C4908700020B7
:10B520000B49087010BD000072000020FA040020D2
:10B53000000C014084000020860000206C000020E8
:10B540008500002075000020800000206F00002092
:10B550007000002010B52A48C07A012839D1294846
:10B560000088002844D12648007B70B14FF48061E8
:10B570002548FCF75CFCB0B10320244908704FF467
:10B5800080612148FCF75CFC0DE04FF480611E48AF
:10B59000FCF74DFC38B903201C4908704FF480615A
:10B5A0001948FCF74FFC1948007808BB4FF40061BC
:10B5B0001548FCF73CFC18B9154800781549087087
:10B5C0004FF400611048FCF73DFC0120124908705F
:10B5D0000EE04FF480610C48FCF729FC18B90C48C8
:10B5E00000780C4908704FF480610748FCF72AFC8A
:10B5F00000200A49087001200949087010BD0000A8
:10B60000FA04002072000020000C01408400002099
:10B61000860000206C000020800000206F000020C9
:10B620007000002010B51648007820B94FF4006172
:10B630001448FCF705FCFFF7E1FE4FF48061114868
:10B64000FCF7F5FB58B11048C07A012807D03C2020
:10B650000E4908804FF480610A48FCF7F1FB4FF473
:10B6600080710B48FCF7ECFB08210948FCF7E8FB6C
:10B67000002008490870084908700849087010BD82
:10B6800084000020000C0140FA0400208200002009
:10B69000000801406F000020700000206D000020B5
:10B6A00000B587B0012144F20400FCF7F1FC03204F
:10B6B0008DF81A0010208DF81B008020ADF81800BE
:10B6C00006A92948FCF7D2FA03208DF81A001820A1
:10B6D0008DF81B004FF40070ADF8180006A9224841
:10B6E000FCF7C4FA48208DF81B004FF48060ADF8D9
:10B6F000180006A91C48FCF7B9FA4FF496400290CE
:10B700000020ADF80C00ADF80E00ADF81000ADF85B
:10B7100014000C20ADF8120002A91448FDF7C0F87F
:10B72000012240F225511148FDF794F8012240F220
:10B7300026610E48FDF78EF801210C48FDF771F8DF
:10B7400025208DF8040000208DF805008DF80600F6
:10B7500001208DF8070001A8FCF726FC8021024893
:10B76000FCF76EFB07B000BD000801400038014047
:10B7700070B5AB48407A022803D0A948407A032824
:10B7800003D10520A749087002E03C20A5490870B4
:10B79000A548007810B9A5480078B0B9A24800784B
:10B7A000012802D1A248007878B19D48407A01284A
:10B7B0000BD0A04800884FF6FF71884205D09D4805
:10B7C000008810B19648408858B9FFF72BFF4FF416
:10B7D00080619948FCF734FB10219848FCF730FB56
:10B7E0001DE18F48807A10B99548008820B110215A
:10B7F0009248FCF727FB03E010219048FCF720FB60
:10B800008748007A10B18648448801E084488488DB
:10B810008348C07A03283ED18148807920448549F5
:10B820000988884202DAFFF723FE05E08148008894
:10B83000A04201DAFFF7F6FE08218048FCF700FB82
:10B840007748807904EB40007A490988884212DA07
:10B850004FF400617848FCF7EAFA60B101207949B9
:10B860000870794800780028BAD14FF48071734885
:10B87000FCF7E8FAD3E06A48807920446D490988EA
:10B880008842ADDD4FF480716C48FCF7D9FA002096
:10B890006C490870C3E06248C07A02283DD1604814
:10B8A0008079201A63490988884202DDFFF752FE39
:10B8B00005E060480088A04201DDFFF7B3FE4FF4C9
:10B8C00080715E48FCF7BCFA55488079A4EB4000D3
:10B8D00058490988884211DD4FF480615648FCF7C9
:10B8E000A6FA58B101205749087057480078002837
:10B8F000C0D108215148FCF7A5FA90E0484880796A
:10B90000201A4C490988884206DA08214B48FCF77E
:10B9100097FA00204B49087081E041488079201A4D
:10B9200044490988884230DD4848007810B1FFF763
:10B9300079FE74E0FFF70EFE4FF480713F48FCF78C
:10B940007FFA3748C07A012805D1C1023A48FCF78E
:10B950006EFA054605E04FF480613748FCF767FA58
:10B9600005462F488079A4EB400032490988884277
:10B9700055DDB5B30120334908703348007880BBEA
:10B9800008212E48FCF75EFA49E0254880792044DA
:10B9900028490988884225DA2D48007810B1FFF738
:10B9A00041FE3CE0FFF764FD08212448FCF748FA1B
:10B9B0001B48807904EB40001E49098888422EDA32
:10B9C0004FF400611C48FCF732FA50B101201D49C8
:10B9D00008701D48007820B94FF480711748FCF7B3
:10B9E00031FA1CE01948007818B112480088A042CA
:10B9F00006DB1748007830B10E480088A04202DD0F
:10BA0000FFF710FE0BE008210C48FCF719FA4FF481
:10BA100080710A48FCF714FA00200A49087070BDCA
:10BA2000FA040020860000205E000020550000205F
:10BA30007400002064000020000C01400008014058
:10BA4000820000206D0000206C0000206F000020AC
:10BA5000700000202DE9F84305460E46174698462B
:10BA6000DDE9084933463A46314628460094FEF758
:10BA700023FE43462A46314628460094FEF71CFE24
:10BA800043463A46414628460094FEF715FE434693
:10BA90003A46314638460094FEF70EFE43463A4693
:10BAA00031462846CDF80090FEF730FDBDE8F8831A
:10BAB00070B5002500240F4E00BF17E0B02141EA09
:10BAC000E400FCF70BFA1020FCF708FA0020FCF762
:10BAD00005FA002505E016F8010BFCF72DFA681CA5
:10BAE000C5B2602DF7DB04F10800C4B2402CE5DDDF
:10BAF00070BD0000A00000201CB51224A01E81B261
:10BB00001348FCF7A3F912490882084610230122C2
:10BB10000021CDE90004AE20FEF7CCF8012802D1C7
:10BB20000C49087002E000200A49087008481023F8
:10BB300001224021CDE90004AE20FEF7BBF8012828
:10BB400002D10449087002E00020024908701CBDBF
:10BB5000FA0400204F00002070B5034601F00706EC
:10BB60000125B540ECB2CD1005EB45050A4E06EBBC
:10BB70004515E85C012A01D1204305E00AB9A0433C
:10BB800002E0022A00D16040CD1005EB4505024ECF
:10BB900006EB4515E85470BDA000002010B591EAF1
:10BBA000030F48BF83F0004300F1B483841A71EBA4
:10BBB000030C05D2121943EB0C03001B61EB0C01C3
:10BBC000DFF824E14FEA1154A4EB135C1EEA430FA3
:10BBD00018BF9EEA445F73D023EA0E03DCF1200E07
:10BBE00021EA045143F4801332D322FA0CFE10EB05
:10BBF0000E0023FA0CFE41EB0E01CCF1200E03FAED
:10BC00000EFE10EB0E0051F10001B1F5801FCCF1DA
:10BC1000200E32D201EB045112FA0EF2BDE81040B0
:10BC200058BF7047401C38BF5FEA420218BF7047D8
:10BC3000002814BF20F0010041F100014FEA410348
:10BC400013F5001F38BF7047A1F1C04100F048BB99
:10BC5000012A43EB0302ACF1200CDCF11F0E32BFD2
:10BC60004FF0000E23FA0CF310EB030041EB0451EC
:10BC7000B4EB115FD0D0A1EB045101F5801149085C
:10BC80005FEA300001EB04510ED350F1000038BFE1
:10BC900012FA0EFE08D1BDE81040C9E7401C38BFBB
:10BCA0005FEA4202CAD1C3E7BDE810404FEA410350
:10BCB00013F5001F38BF7047A1F1C04100F010BB61
:10BCC0009EEA445F08D011EA5E0FBDE8104004BF51
:10BCD00001F0004100207047BDE8104070B500F051
:10BCE000B1FA00BF64FBBE3E0000E0FF02494FF026
:10BCF000000000F0F1BB00BF0000F87F491058BF02
:10BD0000C1F140415B1058BFC3F140438B42EFF398
:10BD1000008070472DE9C04130B4DFF8A0C23CEA92
:10BD2000111418BF3CEA131400F0EC8081EA0305FB
:10BD30001CEA111444EAD57418BF1CEA131500F06C
:10BD4000C780A4EB05044FF0004545EAC12145EA50
:10BD5000C32341EA505143EA525304F17F7499429C
:10BD600004F500344FEAC0204FEAC22208BF9042D7
:10BD700000F09C804FEA13650FF24016765D4FEAA3
:10BD8000134506FB05F7C7F1807706FB07F74FEA77
:10BD9000D737A7FB03687642C8F58038A7FB06CEE5
:10BDA00038BFA8F1010807FB08E64FF0000EA6FB1C
:10BDB000028CE6FB03CEDCF1000CCEF1004E38BF66
:10BDC000AEF1010EA6FB0C584FF000074FF0000536
:10BDD000E6FB0E87A1FB08C6A0FB07CE16EB0E06FE
:10BDE00045F10005E1FB076515F1E04E7EBFA4F5C6
:10BDF00080345FEA46066D4116F1800745F1000583
:10BE00004FEA17274FEA066647EA0567A6F1DE46BE
:10BE1000B6F1805F4FEA15251FD9384624F0010C92
:10BE200005EBC471BCF1FE6F01EB0C1102D8F0BC44
:10BE3000BDE8008124425CBF01F5801E9EEAC47FFC
:10BE400002D4F0BCBDE80081244238D4F0BCA1F19A
:10BE5000C041BDE8004100F043BA4FEAD22242EAB5
:10BE600043524FEAD323A7FB02864FEAD02040EA91
:10BE7000415007FB03661EEA0E0F4FEAD12105FB76
:10BE8000026658BFA6EB0056B6EB00564FEA520EBC
:10BE90004EEAC37E18EB0E0E56EB530EBDD518EBD3
:10BEA00002085E417F1C55F10005B6E74FF480158E
:10BEB0004FF000074FF000064FF00008ADE7F0BC70
:10BEC0004FF0000001F1C04101F00041BDE80081E8
:10BED00011EA0C1F0CEA131500D00CE013EA0C1F3A
:10BEE00000F025804FF00000F0BC81EA030101F072
:10BEF0000041BDE80081F0BCBDE8004181EA0301DA
:10BF000000F0EEB9F0BCBDE8004170B500F09AF960
:10BF1000097EFC3E00F007B881EA03014FF0000003
:10BF200001F00041704781EA030100F0D9B9F0BC8B
:10BF3000BDE800414FF0000021497047FFFDFBF9CB
:10BF4000F7F5F4F2F0EEEDEBE9E8E6E4E3E1E0DE4C
:10BF5000DDDBDAD8D7D5D4D3D1D0CFCDCCCBCAC8BE
:10BF6000C7C6C5C4C2C1C0BFBEBDBCBBBAB9B8B7E5
:10BF7000B6B5B4B3B2B1B0AFAEADACABAAA9A8A8D8
:10BF8000A7A6A5A4A3A3A2A1A09F9F9E9D9C9C9BA6
:10BF90009A99999897979695959493939291919051
:10BFA0008F8F8E8E8D8C8C8B8B8A898988888787E2
:10BFB0008685858484838382828181800000FF0757
:10BFC0000000F87F51EA030C17D41CF5801F58BFFE
:10BFD000BCF5801F00F10680994218BF704708BF6A
:10BFE0009042704707D711F5801F58BF13F5801F87
:10BFF00019D499427047894270471CF5801F08D5B3
:10C00000BCF5801FF7D58B4218BF704708BF82422E
:10C0100070474FF4001C1CEB410F38BF1CEB430F63
:10C0200001D28B42704770B500F00CF992244900A0
:10C030004FF000514FF08053FFF760BE4FEA4103CD
:10C040004FEA5353A3F58063D3F11E03C8BFD3F166
:10C05000210C0CDD4FF0004242EAC12242EA50526C
:10C0600032FA03FC8CEAE17CACEBE1707047102BF8
:10C07000C4BF0020704703F5787CBCF1FF3F04D0BB
:10C080006FF0004282EA2100704770B500F0DAF8E4
:10C090004992248000207047F2E710F0004248BF28
:10C0A0004042B0FA80F310FA03F10AD0C3F11D0345
:10C0B00003F580634FEA415002EB035202EBD121BA
:10C0C00070474FF000007047B0FA80F310FA03F1A8
:10C0D0000AD0C3F11D0303F580634FEA41504FEAD4
:10C0E000035202EBD12170474FF00000704700006F
:10C0F000DFF848C170B51CEA111E1EBF1CEA1315FB
:10C100009EEA0C0F95EA0C0F00F06F8081EA0304A1
:10C1100023EA4C134EEAD47E21EA4C1141F48011FB
:10C1200043F48013AE44A1FB024CA0FB0365AEF1C7
:10C130007F7E361955EB0C05A1FB034C4CF1000337
:10C14000A0FB021C16EB0C06654153F100030942EB
:10C1500018BF46F0010613F4007F0BD14FEA0331FC
:10C160004FEA0530340341EA155140EA16506FF0AA
:10C1700003020AE04FEAC3214FEAC520F40241EA74
:10C18000555140EA56506FF0020202EB2E4201EB8D
:10C19000025585EACE710AD05FEA440C18BF24F03C
:10C1A000004450F1000041F1000120EAD47040F257
:10C1B000FE7C624500D270BDA84214BF4FF080449F
:10C1C0004FF04044002E08BF0024BEF1806FA8BF8E
:10C1D000A1F1C041BDE8704080F282804FF00000C4
:10C1E00001F1C04101F0004170479EEA0C0F0CEADA
:10C1F000131518BF95EA0C0F06D04FF0000081EA26
:10C20000030E0EF0004170BD00F01CF88900013EE5
:10C2100000F007B800F009B84FEA430C5FEA5C5C35
:10C2200008D081EA030100F05BB84FEA410C5FEAF5
:10C230005C5CF6D14FF00000014970470000FF0739
:10C240000000F87F0EF1020E2EF0030E5EF8046B74
:10C25000364205D4012A43EB030515F5001F12D819
:10C26000012841EB010C1CF5001F0CD80ED14FEA40
:10C27000D17C15F5001F0CEB4C0C0CF1020C08BF27
:10C280004CEBD37C04E04FF0080C01E04FEAD37C88
:10C290000CEB4C0526FA05F606F00706B6F1040C81
:10C2A00006D20EEB860CBDE870404CF0010C6047E6
:10C2B000DFE80CF0090B02024FF000414FF00000E4
:10C2C000A1F5002170BD19461046012851EB01046B
:10C2D00018BFD4F5001484BF002001F0004170BDE8
:10C2E0000808A0F500114FEA3101704791EA030FE9
:10C2F00010B581F000413FF559AC83F0004300F0E8
:10C3000009B8000010B591EA030F48BF83F000435D
:10C310003FF54CAC841A71EB030C07D212198CF068
:10C32000004C43EB0C03001B61EB0C01DFF8A4E1B4
:10C330004FEA1154A4EB135C1EEA430F18BF9EEAA8
:10C34000445F00F0B08023EA6E03524221EA0451B8
:10C35000C3EB6E0338BF5B1EDCF1200E25D322FA3F
:10C360000CFE10EB0E0043FA0CFE41EB0E01CCF17B
:10C37000200E03FA0EFE10EB0E0051F10001CCF17D
:10C38000200E29D412FA0EF201EB0451BDE8104040
:10C3900058BF7047401C1CBFB2F1004F70470028C7
:10C3A0000CBF491C20F00100704712EB020E43EB5A
:10C3B000030218BF4FF0010E4EEA4202ACF1200C0E
:10C3C000DCF11E0E54D943FA0CFE10EB0E0051F1B5
:10C3D000FF31CCF11E0ED5D50EF1010E12FA0EFE74
:10C3E000404141EB010101EB445C5FEA5C5C10D928
:10C3F00010EBDE7001EB045138BFBEF1004FBDE819
:10C40000104018BF704700280CBF491C20F00100E5
:10C41000704730D24FEAD42C11F5001124F4006497
:10C420001BD0B1FA81F20B3AA41AA41ED2F1200358
:10C43000914030FA03F31943904001EBCC71002C8A
:10C4400001EB0451BDE81040A8BF704701F1C041A5
:10C450004FF0000001F000417047B0FA80F310FA8D
:10C4600003F100D110BDE41A173C4805C90AE4E7FE
:10C4700001EB045110BD491001EB0451BDE810401F
:10C480004FEA300002E04FF0000170474A0008BF59
:10C490000042F8D0B2F5001F28BF704701F00041FC
:10C4A0004FF0000070479EEA445F07D011EA5E0F2C
:10C4B000BDE8104004BF002100207047BDE81040D7
:10C4C00070B5FFF7BFFE00BF40DFF63E83F00041CE
:10C4D000104670470000E0FF0CF00F03092B08BF67
:10C4E000082000F059800A2B0BD0082B18BF70478A
:10C4F00008BF1CF0400F0AD04FF000004FF00001C1
:10C5000070471CF0400F18BF4FF0004070471CF000
:10C51000100F08D020F0704300F07F4242EAD301B0
:10C520004FEA4370704700F0604021F07F4242EADA
:10C53000000201F07F4040EA727070474FF0FF0C3C
:10C540004CF4E06C1CEA11531CBF9CEA030C9445AC
:10C55000C2BFDA4201EB02517047002B0DD0BCF193
:10C56000000F0FD0002A01F00041A4BF41F0E041CC
:10C5700041F07F614FF00000704701F000414FF043
:10C580000000704750EA01334FF09B0C18BF4CF08D
:10C59000806C7FF4ABAB70471CF4801F11D01CF48F
:10C5A000E02F03D06FEACC31490070474FF0405084
:10C5B000EFF3008222F0704242EA000282F3008828
:10C5C00070474FF0000070470000000000000000BE
:10C5D00020202020200020004848480000000000C3
:10C5E0005050F850F85050002078A07028F02000EB
:10C5F000C0C81020409818006090A040A890680023
:10C60000602040000000000010204040402010004A
:10C610004020101010204000005020F82050000052
:10C62000002020F8202000000000000000602040D2
:10C63000000000F800000000000000000060600042
:10C640000008102040800000708898A8C8887000FA
:10C650002060202020207000708808304080F80082
:10C66000708808300888700010305090F810100062
:10C67000F880F00808887000304080F088887000EA
:10C68000F80810204040400070888870888870004A
:10C6900070888878081060000060600060600000AA
:10C6A00000006060006020401020408040201000AA
:10C6B0000000F800F80000008040201020408000BA
:10C6C000708808102000200070880868A8A87000F2
:10C6D000708888F888888800F08888F08888F0005A
:10C6E0007088808080887000E09088888890E00062
:10C6F000F88080F08080F800F88080F080808000F2
:10C700007088808098887800888888F88888880071
:10C710007020202020207000381010101090600031
:10C720008890A0C0A0908800808080808080F800E1
:10C7300088D8A8A8888888008888C8A89888880089
:10C740007088888888887000F08888F080808000F1
:10C7500070888888A8906800F08888F0A090880089
:10C760007088807008887000F82020202020200029
:10C770008888888888887000888888888850200001
:10C78000888888A8A8A850008888502050888800E9
:10C790008888885020202000F80810204080F80069
:10C7A0007040404040407000008040201008000071
:10C7B0007010101010107000205088000000000051
:10C7C00000000000000000F8402010000000000001
:10C7D00000007008788878008080B0C88888F000F1
:10C7E0000000708080887000080868988888780049
:10C7F00000007088F8807000304840E04040400001
:10C8000000007888887808708080B0C888888800A0
:10C810002000602020207000100030101010906068
:10C82000808090A0C0A09000602020202020700078
:10C830000000D0A8888888000000B0C888888800D8
:10C8400000007088888870000000F08888F0808080
:10C8500000007888887808080000B0C880808000D0
:10C86000000078807008F0004040E0404048300010
:10C870000000888888986800000088888850200018
:10C8800000008888A8A85000000088502050880028
:10C8900000008888887808700000F8102040F800B0
:10C8A00010202040202010002020202020202000C8
:10C8B0004020201020204000689000000000000070
:10C8C0000000000000000000183C3C181800180090
:10C8D00066662400000000006C6CFE6CFE6C6C0050
:10C8E000183E603C067C180000C6CC183066C600B6
:10C8F000386C3876DCCC7600181830000000000068
:10C900000C18303030180C0030180C0C0C1830009B
:10C9100000663CFF3C6600000018187E18180000F6
:10C9200000000000001818300000007E0000000029
:10C930000000000000181800060C183060C08000CD
:10C94000386CC6C6C66C38001838181818187E001F
:10C950007CC6061C3066FE007CC6063C06C67C0013
:10C960001C3C6CCCFE0C1E00FEC0C0FC06C67C004D
:10C970003860C0FCC6C67C00FEC60C1830303000E3
:10C980007CC6C67CC6C67C007CC6C67E060C78000B
:10C9900000181800001818000018180000181830A7
:10C9A000060C1830180C060000007E00007E000007
:10C9B0006030180C183060007CC60C181800180085
:10C9C0007CC6DEDEDEC07800386CC6FEC6C6C60099
:10C9D000FC66667C6666FC003C66C0C0C0663C00C7
:10C9E000F86C6666666CF800FE6268786862FE0045
:10C9F000FE6268786860F0003C66C0C0CE663A00AF
:10CA0000C6C6C6FEC6C6C6003C18181818183C0094
:10CA10001E0C0C0CCCCC7800E6666C786C66E600DC
:10CA2000F06060606266FE00C6EEFEFED6C6C6001E
:10CA3000C6E6F6DECEC6C6007CC6C6C6C6C67C0046
:10CA4000FC66667C6060F0007CC6C6C6C6CE7C0E06
:10CA5000FC66667C6C66E6003C6630180C663C0042
:10CA60007E7E5A1818183C00C6C6C6C6C6C67C00CC
:10CA7000C6C6C6C6C66C3800C6C6C6D6D6FE6C00CC
:10CA8000C6C66C386CC6C6006666663C18183C00A4
:10CA9000FEC68C183266FE003C30303030303C0030
:10CAA000C06030180C0602003C0C0C0C0C0C3C0056
:10CAB00010386CC60000000000000000000000FFFD
:10CAC00030180C00000000000000780C7CCC7600D0
:10CAD000E0607C666666DC0000007CC6C0C67C0048
:10CAE0001C0C7CCCCCCC760000007CC6FEC07C004C
:10CAF0003C6660F86060F000000076CCCC7C0CF8FE
:10CB0000E0606C766666E6001800381818183C007D
:10CB1000060006060666663CE060666C786CE60019
:10CB20003818181818183C000000ECFED6D6D600AD
:10CB30000000DC666666660000007CC6C6C67C0037
:10CB40000000DC66667C60F0000076CCCC7C0C1EBD
:10CB50000000DC766060F00000007EC07C06FC0017
:10CB60003030FC3030361C000000CCCCCCCC760011
:10CB70000000C6C6C66C38000000C6D6D6FE6C00E3
:10CB80000000C66C386CC6000000C6C6C67E06FC37
:10CB900000007E4C18327E000E18187018180E0017
:10CBA00018181818181818007018180E181870008F
:10CBB00076DC0000000000000C1000000000000007
:10CBC00060100000000000007C82000000000000F7
:10CBD000C600000000000000728C00000000000091
:10CBE0000000381818183C00386C6C7866666CC009
:10CBF00018003C667E6666003000780C7CCC7600BF
:10CC00001E78989EF8989E007C6666F666667C00A4
:10CC1000F0607C66667C60F00000CC327EB0EC0098
:10CC20006830580C7EC67C0070303C363C30780052
:10CC30003A6CCED6E66CB80000027CCED6E67C809C
:10CC400000007CC6FEC6C6000000FE607C60FE00E0
:10CC500000003C1818183C0000007CC6C6C67C00CA
:10CC60000000C6C6C6C67C000000E6F6DECEC600E2
:10CC7000180018183C3C18003000303060C67C00AA
:10CC80000C10000000000000601000000000000018
:10CC90003844000000000000C60000000000000052
:10CCA000728C000000000000000000000000001076
:10CCB000000000000000000000107CD0D0D67C10E6
:10CCC0001C30307830325C00000044382838440092
:10CCD00044287C107C1010003030300030303000A0
:10CCE0003840304830087000C600000000000000E6
:10CCF0007E425A5E5A427E0038043C4438000000AE
:10CD000000366CD86C3600000000007C0404000083
:10CD10000000007C000000007C4454444C547C0023
:10CD20007C000000000000003048300000000000DF
:10CD300010107C1010007C0060902040F00000007B
:10CD4000E0106010E00000000E182000000000005D
:10CD50000000666666667CC07ED4D47414143E00FF
:10CD6000000000181800000040C04040E000000033
:10CD70003C6666663C00000000D86C366CD800004B
:10CD8000848890A44C941E04848890AC5284081E1D
:10CD9000C0204024CC141E0400663C183C660000F1
:10CDA0000018007E00180000103070FC7030100079
:10CDB000203038FC38302000002070F8202000009F
:10CDC000002020F87020000000082868F86020008B
:10CDD0000606060C8CD87830000000000000000029
:10CDE00000000000003078787830300030300000EB
:10CDF000006666662400000000000000006C6CFE07
:10CE00006C6C6CFE6C6C000030307CC0C0780C0C1C
:10CE1000F8303000000000C4CC183060CC8C00002A
:10CE20000070D8D870FADECCDC76000000303030EC
:10CE30006000000000000000000C183060606030EE
:10CE4000180C0000006030180C0C0C18306000004A
:10CE5000000000663CFF3C66000000000000001877
:10CE6000187E1818000000000000000000000000FC
:10CE7000383860000000000000FE000000000000E4
:10CE8000000000000000000038380000000002062A
:10CE90000C183060C0800000007CC6CEDED6F6E6FE
:10CEA000C67C0000001030F03030303030FC000024
:10CEB0000078CCCC0C183060CCFC00000078CC0C96
:10CEC0000C380C0CCC780000000C1C3C6CCCFE0C1C
:10CED0000C1E000000FCC0C0C0F80C0CCC78000098
:10CEE000003860C0C0F8CCCCCC78000000FEC6C6CC
:10CEF000060C1830303000000078CCCCEC78DCCC5C
:10CF0000CC7800000078CCCCCC7C181830700000B5
:10CF100000000038380000383800000000000038F9
:10CF20003800003838183000000C183060C060300D
:10CF3000180C0000000000007E007E0000000000D1
:10CF4000006030180C060C18306000000078CC0C23
:10CF50001830300030300000007CC6C6DEDEDEC097
:10CF6000C07C0000003078CCCCCCFCCCCCCC000019
:10CF700000FC6666667C666666FC0000003C66C671
:10CF8000C0C0C0C6663C000000F86C666666666697
:10CF90006CF8000000FE6260647C646062FE000069
:10CFA00000FE6662647C646060F00000003C66C65F
:10CFB000C0C0CEC6663E000000CCCCCCCCFCCCCCF5
:10CFC000CCCC000000783030303030303078000089
:10CFD000001E0C0C0C0CCCCCCC78000000E6666C6F
:10CFE0006C786C6C66E6000000F060606060626601
:10CFF00066FE000000C6EEFEFED6C6C6C6C600002F
:10D0000000C6C6E6F6FEDECEC6C6000000386CC618
:10D01000C6C6C6C66C38000000FC6666667C6060EA
:10D0200060F0000000386CC6C6C6CEDE7C0C1E0068
:10D0300000FC6666667C6C6666E600000078CCCC18
:10D04000C07018CCCC78000000FCB43030303030E8
:10D050003078000000CCCCCCCCCCCCCCCC78000050
:10D0600000CCCCCCCCCCCCCC7830000000C6C6C632
:10D07000C6D6D66C6C6C000000CCCCCC783078CCAA
:10D08000CCCC000000CCCCCCCC7830303078000058
:10D0900000FECE9818306062C6FE0000003C3030C2
:10D0A00030303030303C0000000080C06030180C60
:10D0B00006020000003C0C0C0C0C0C0C0C3C00009C
:10D0C00010386CC6000000000000000000000000E6
:10D0D000000000000000FF003030180000000000D9
:10D0E0000000000000000000780C7CCCCC76000032
:10D0F00000E060607C66666666DC000000000000A0
:10D1000078CCC0C0CC780000001C0C0C7CCCCCCC03
:10D11000CC7600000000000078CCFCC0CC78000089
:10D1200000386C6060F8606060F000000000000093
:10D1300076CCCCCC7C0CCC7800E060606C766666FB
:10D1400066E600000018180078181818187E00000D
:10D15000000C0C003C0C0C0C0CCCCC7800E060609B
:10D16000666C786C66E600000078181818181818B5
:10D17000187E000000000000FCD6D6D6D6C60000FF
:10D1800000000000F8CCCCCCCCCC000000000000AB
:10D1900078CCCCCCCC78000000000000DC66666661
:10D1A000667C60F00000000076CCCCCCCC7C0C1E01
:10D1B00000000000EC6E766060F0000000000000EF
:10D1C00078CC6018CC78000000002060FC606060C3
:10D1D0006C38000000000000CCCCCCCCCC76000039
:10D1E00000000000CCCCCCCC783000000000000067
:10D1F000C6C6D6D66C6C000000000000C66C38387D
:10D200006CC6000000000000666666663C0C18F004
:10D2100000000000FC8C1860C4FC0000001C3030D2
:10D2200060C06030301C0000001818181800181872
:10D230001818000000E03030180C183030E0000002
:10D240000073DACE000000000000000000000010B3
:10D25000386CC6C6FE0000000000000000000000A0
:10D2600000000000000000000000183C3C3C1818C2
:10D270001800181800000000006666662400000010
:10D2800000000000000000000000006C6CFE6C6CF0
:10D290006CFE6C6C0000000018187CC6C2C07C06D6
:10D2A0000686C67C1818000000000000C2C60C18D4
:10D2B0003060C686000000000000386C6C3876DCF8
:10D2C000CCCCCC7600000000003030306000000094
:10D2D000000000000000000000000C18303030306A
:10D2E0003030180C00000000000030180C0C0C0C42
:10D2F0000C0C1830000000000000000000663CFF2D
:10D300003C66000000000000000000000018187ECD
:10D3100018180000000000000000000000000000DD
:10D32000001818183000000000000000000000FE87
:10D3300000000000000000000000000000000000ED
:10D3400000001818000000000000000002060C1881
:10D350003060C080000000000000386CC6C6C6C641
:10D36000C6C66C380000000000001838781818187D
:10D370001818187E0000000000007CC6060C18304B
:10D3800060C0C6FE0000000000007CC606063C0629
:10D390000606C67C0000000000000C1C3C6CCCFEA5
:10D3A0000C0C0C1E000000000000FEC0C0C0FC06FB
:10D3B0000606C67C0000000000003860C0C0FCC645
:10D3C000C6C6C67C000000000000FEC606060C189B
:10D3D000303030300000000000007CC6C6C67CC67D
:10D3E000C6C6C67C0000000000007CC6C6C67E061D
:10D3F00006060C780000000000000000181800006D
:10D4000000181800000000000000000018180000BC
:10D410000018183000000000000000060C183060F2
:10D4200030180C060000000000000000007E000024
:10D430007E000000000000000000006030180C06B4
:10D440000C1830600000000000007CC6C60C1818E4
:10D4500018001818000000000000007CC6C6DEDEC0
:10D46000DEDCC07C00000000000010386CC6C6FE88
:10D47000C6C6C6C6000000000000FC6666667C6684
:10D48000666666FC0000000000003C66C2C0C0C0CA
:10D49000C0C2663C000000000000F86C666666666C
:10D4A00066666CF8000000000000FE66626878683E
:10D4B000606266FE000000000000FE666268786838
:10D4C000606060F00000000000003C66C2C0C0DE8A
:10D4D000C6C6663A000000000000C6C6C6C6FEC644
:10D4E000C6C6C6C60000000000003C181818181870
:10D4F0001818183C0000000000001E0C0C0C0C0C4E
:10D50000CCCCCC78000000000000E666666C787831
:10D510006C6666E6000000000000F060606060601D
:10D52000606266FE000000000000C6EEFEFED6C689
:10D53000C6C6C6C6000000000000C6E6F6FEDECE87
:10D54000C6C6C6C60000000000007CC6C6C6C6C669
:10D55000C6C6C67C000000000000FC6666667C60F3
:10D56000606060F00000000000007CC6C6C6C6C651
:10D57000C6D6DE7C0C0E00000000FC6666667C6C85
:10D58000666666E60000000000007CC6C660380CD7
:10D5900006C6C67C0000000000007E7E5A181818DF
:10D5A0001818183C000000000000C6C6C6C6C6C653
:10D5B000C6C6C67C000000000000C6C6C6C6C6C6F9
:10D5C000C66C3810000000000000C6C6C6C6D6D61D
:10D5D000D6FEEE6C000000000000C6C66C7C383839
:10D5E0007C6CC6C6000000000000666666663C18DB
:10D5F0001818183C000000000000FEC6860C183009
:10D6000060C2C6FE0000000000003C303030303008
:10D610003030303C0000000000000080C0E0703876
:10D620001C0E06020000000000003C0C0C0C0C0C50
:10D630000C0C0C3C0000000010386CC60000000010
:10D6400000000000000000000000000000000000DA
:10D650000000000000FF00000030180C0000000077
:10D6600000000000000000000000000000780C7CBA
:10D67000CCCCCC76000000000000E06060786C66E6
:10D680006666667C0000000000000000007CC6C0EA
:10D69000C0C0C67C0000000000001C0C0C3C6CCC20
:10D6A000CCCCCC760000000000000000007CC6FE60
:10D6B000C0C0C67C0000000000001C36323078304C
:10D6C0003030307800000000000000000076CCCC44
:10D6D000CCCCCC7C0CCC78000000E060606C766632
:10D6E000666666E60000000000001818003818188A
:10D6F0001818183C0000000000000606000E060680
:10D700000606060666663C000000E06060666C780F
:10D71000786C66E600000000000038181818181829
:10D720001818183C000000000000000000ECFED6B5
:10D73000D6D6D6C6000000000000000000DC6666F9
:10D74000666666660000000000000000007CC6C639
:10D75000C6C6C67C000000000000000000DC666653
:10D760006666667C6060F000000000000076CCCC4D
:10D77000CCCCCC7C0C0C1E000000000000DC7666DB
:10D78000606060F00000000000000000007CC660E7
:10D79000380CC67C000000000000103030FC303037
:10D7A0003030361C000000000000000000CCCCCC63
:10D7B000CCCCCC76000000000000000000C6C6C63D
:10D7C000C6C66C38000000000000000000C6C6D6C7
:10D7D000D6D6FE6C000000000000000000C66C38C9
:10D7E00038386CC6000000000000000000C6C6C645
:10D7F000C6C6C67E060CF8000000000000FECC186D
:10D800003060C6FE0000000000000E1818187018E6
:10D810001818180E00000000000018181818181822
:10D8200018181818000000000000701818180E18BA
:10D8300018181870000000000076DC0000000000DE
:10D84000000000000000000000001C30000000008C
:10D850000000000000000000000070180000000040
:10D8600000000000000000000010386C0000000004
:10D87000000000000000000000C6C600000000001C
:10D8800000000000000000000076DC000000000046
:10D890000000000000000000000000000038181820
:10D8A0001818183C000000000000386C6C6C786C94
:10D8B0006666666C60C00000102810007CC6C6FE5C
:10D8C000C6C6C6C6000000000030483000780C7C98
:10D8D000CCCCCC760000000000001E7AD8D8D8FE50
:10D8E000D8D8DADE000000000000FC666666F6F6B6
:10D8F000666666FC000000000000F0607C666666FC
:10D90000667C60F0000000000000000000CC323EA9
:10D9100070B0B26C000000000000D060B0187CC68F
:10D92000C6C6C67C000000000000E06060786C6C39
:10D93000786060F00000000000007CC6CECED6D635
:10D94000E6E6C67C0000000000000000003A44CE7D
:10D95000D6E644B800000000000000386CC6C6FEE1
:10D96000C6C6C6C600000000000000FE66626878F9
:10D97000686266FE000000000000003C18181818DD
:10D980001818183C000000000000007CC6C6C6C67F
:10D99000C6C6C67C00000000000000C6C6C6C6C6DB
:10D9A000C6C6C67C00000000000000C6E6F6FEDE2B
:10D9B000CEC6C6C6000000000000181800181818CF
:10D9C0003C3C3C180000000000003030003030309B
:10D9D00060C6C67C000000001C3000000000000093
:10D9E00000000000000000007018000000000000AF
:10D9F0000000000000000000386C00000000000083
:10DA00000000000000000000C6C60000000000008A
:10DA1000000000000000000076DC000000000000B4
:10DA200000000000000000000000000000000000F6
:10DA3000000000001830000000000000000000009E
:10DA4000000000000000000000000010107CD0D09A
:10DA5000D0D0D67C1010000000001C303030783060
:10DA60003030325C0000000000000000423C242402
:10DA70003C420000000000000000663C187E1818C0
:10DA80007E18181800000000000018181818000070
:10DA9000181818180000000000003C646038444466
:10DAA000380C4C780000000000C6C60000000000E2
:10DAB0000000000000000000000000007E425A5EEE
:10DAC0005A427E00000000000000700878888874C8
:10DAD00000000000000000000000000000366CD8CC
:10DAE0006C3600000000000000000000000000FC98
:10DAF0000404000000000000000000000000007CA2
:10DB00000000000000000000000000007C445444BD
:10DB10004C547C0000000000FE00000000000000EB
:10DB200000000000000000000070D888D8700000DD
:10DB300000000000000000000000000010107C1039
:10DB400010007C0000000000788C0C183060FC0095
:10DB50000000000000000000788C0C780C8C78002D
:10DB60000000000000000000000E1820000000006F
:10DB70000000000000000000000000000066666673
:10DB80006666667C6060C00000007ED4D4D47414E5
:10DB90001414143E0000000000000000000038389B
:10DBA000380000000000000060E060606060F0008D
:10DBB000000000000000000000003C6666663C00BB
:10DBC00000000000000000000000000000D86C36DB
:10DBD0006CD8000000000000000040C04448102441
:10DBE0004C941E0400000000000040C04448102C6B
:10DBF0005284081E000000000000C0204428D024E9
:10DC00004C941E04000000000000000000663C1858
:10DC10003C66000000000000000000001818007EB4
:10DC2000001818000000000000000000000818386C
:10DC30007FFF7F3818080000000000000010181C4B
:10DC4000FEFFFE1C1810000000000000000010384D
:10DC50007CFE3838383800000000000000003838FA
:10DC60003838FE7C38100000000000060606061654
:10DC7000367EFE7C30100000000000000000030330
:10DC800006060CCC78380000000000000000000000
:10DC90000000000000000000000000000000000084
:10DCA0000000000000000000000000000000000074
:10DCB0000000000000000000000000000000000064
:10DCC0003800380038003800380038003800380094
:10DCD0003800100010000000380038003800000044
:10DCE0000000000000000000000000000000000034
:10DCF0007380738073807380738000000000000065
:10DD00000000000000000000000000000000000013
:10DD10000000000000000000000000000000000003
:10DD20000C600C600C6018C0FFF0FFF018C039C028
:10DD30003180FFF0FFF031807380630063000000EA
:10DD400000000000000000000000000000000600CD
:10DD50001F803FC076E076E076007E003F001FC067
:10DD600007E006E006E076E076E03FC01F800600B0
:10DD7000060000000000000000000000000000009D
:10DD80003C187E3866306630666066607EC03CC097
:10DD9000019E01BF03B3033303330633063F0C1E5A
:10DDA0000000000000000000000000000000000073
:10DDB00007800FC01CE01CE01EE00FC00F801F801A
:10DDC0003F9C71FC71F870F079FC3FFE1F8C0000E5
:10DDD0000000000000000000000000000000000043
:10DDE0007000700070007000700000000000000003
:10DDF0000000000000000000000000000000000023
:10DE00000000000000000000000000000000000012
:10DE10000C00180018003800380070007000700006
:10DE20007000700070007000700030003800380022
:10DE3000180018000C0000000000000000000000A6
:10DE4000600030003000380038001C001C001C004E
:10DE50001C001C001C001C001C00180038003800AE
:10DE600030003000600000000000000000000000F2
:10DE700018001800DB00FF001C003C0066002400B6
:10DE80000000000000000000000000000000000092
:10DE90000000000000000000000000000000000082
:10DEA0000000000007000700070007007FF07FF078
:10DEB0007FF00700070007000700000000000000D7
:10DEC0000000000000000000000000000000000052
:10DED0000000000000000000000000000000000042
:10DEE00000000000000000007000700070001000D2
:10DEF0003000600000000000000000000000000092
:10DF00000000000000000000000000000000000011
:10DF10007E007E007E000000000000000000000087
:10DF200000000000000000000000000000000000F1
:10DF300000000000000000000000000000000000E1
:10DF40000000000000000000700070007000000081
:10DF500000000000000000000000000000000000C1
:10DF60000C000C00180018001800380030003000B9
:10DF700030006000600060006000C000C000000071
:10DF80000000000000000000000000000000000091
:10DF90000F003FC039C070E070E070E070E070E0EA
:10DFA00070E070E070E070E039C03FC00F0000002A
:10DFB0000000000000000000000000000000000061
:10DFC0000380038007801F803F803B802380038085
:10DFD00003800380038003800380038003800000AC
:10DFE0000000000000000000000000000000000031
:10DFF0001F803FC079E070E000E000E001C003C096
:10E0000007800F001E001C0038007FE07FE000004A
:10E010000000000000000000000000000000000000
:10E020001F003F8071C071C001C003C00F800F800E
:10E0300001C000E000E070E079C03FC01F000000B8
:10E0400000000000000000000000000000000000D0
:10E050000380078007800F800F801B803380338010
:10E060006380C380FFE0FFE0038003800380000043
:10E0700000000000000000000000000000000000A0
:10E080001FC01FC03800380038003F807FC071E0DB
:10E0900000E000E000E070E079C03FC01F00000039
:10E0A0000000000000000000000000000000000070
:10E0B0000F803FC039E07080700077807FC079C0EA
:10E0C00070E070E070E070E039C03FC00F00000009
:10E0D0000000000000000000000000000000000040
:10E0E0007FE07FE000E001C00380038007000700BD
:10E0F0000E000E000E001C001C001C001C00000086
:10E10000000000000000000000000000000000000F
:10E110001F803FC079E070E070E039C01F801F8031
:10E1200039C070E070E070E079E03FC01F8000000F
:10E1300000000000000000000000000000000000DF
:10E140000F003FC039C070E070E070E070E039E06F
:10E150003FE01EE000E030E079C03FC01F0000005B
:10E1600000000000000000000000000000000000AF
:10E1700000000000000000003800380038000000F7
:10E1800000000000000000003800380038000000E7
:10E19000000000000000000000000000000000007F
:10E1A00000000000000000003800380038000000C7
:10E1B00000000000000000003800380038000800AF
:10E1C0001800300000000000000000000000000007
:10E1D00000000000002000E007E01F807C007000CD
:10E1E0007E001FC007E000E00020000000000000EB
:10E1F000000000000000000000000000000000001F
:10E2000000000000000000007FE07FE07FE00000F1
:10E2100000007FE07FE07FE00000000000000000E1
:10E2200000000000000000000000000000000000EE
:10E2300000000000400070007E001F8003E000E04E
:10E2400007E03F807E0070004000000000000000FA
:10E2500000000000000000000000000000000000BE
:10E260000F803FE078F07070007000F001E003C0B4
:10E2700007800700070000000700070007000000F4
:10E28000000000000000000000000000000000008E
:10E2900003E007F00F1C1C0E19CE33E636666666E7
:10E2A0006666666666666666666663FE31BE380EDC
:10E2B0001C1C0F3C07F003E0000000000000000001
:10E2C00007C007C007C00EE00EE00EE01C701C7017
:10E2D00038383FF83FF87FFC701C701CE00E0000DF
:10E2E000000000000000000000000000000000002E
:10E2F0003FE03FF03FF83838383838383FF03FF0EB
:10E300003FF8381C381C381C3FFC3FF83FF0000039
:10E3100000000000000000000000000000000000FD
:10E3200007C01FF03FF83C3C781870007000700088
:10E330007000700078183C3C3FF81FF007C00000E8
:10E3400000000000000000000000000000000000CD
:10E350003FE03FF03FF83838383C381C381C381C58
:10E36000381C381C381C38383FF83FF03FC00000DC
:10E37000000000000000000000000000000000009D
:10E380003FF83FF83FF83800380038003FF03FF0E2
:10E390003FF03800380038003FF83FF83FF8000001
:10E3A000000000000000000000000000000000006D
:10E3B0003FF03FF03FF03800380038003FE03FE0EA
:10E3C0003FE03800380038003800380038000000DE
:10E3D000000000000000000000000000000000003D
:10E3E00003E00FF81FFC3C1E780C7000700070FEFC
:10E3F00070FE70FE380E3C1E1FFE0FFC03E0000096
:10E40000000000000000000000000000000000000C
:10E410007038703870387038703870387FF87FF81E
:10E420007FF8703870387038703870387038000085
:10E4300000000000000000000000000000000000DC
:10E4400003800380038003800380038003800380B4
:10E450000380038003800380038003800380000027
:10E4600000000000000000000000000000000000AC
:10E4700001C001C001C001C001C001C001C001C094
:10E4800001C0E1C0E1C0F1C07FC07F801E0000007C
:10E49000000000000000000000000000000000007C
:10E4A000383C387838F038E039C03B803FC03FC056
:10E4B0003EE03CE0387038383838381C381C0000F2
:10E4C000000000000000000000000000000000004C
:10E4D000380038003800380038003800380038007C
:10E4E00038003800380038003FF03FF03FF00000BF
:10E4F000000000000000000000000000000000001C
:10E500007C1F7E3F7E3F7637763776377777777713
:10E510007367736773E773E773E771C771C70000C9
:10E5200000000000000000000000000000000000EB
:10E530007038783878387C387E3876387738733861
:10E5400073B871B871F870F870F8707870380000AE
:10E5500000000000000000000000000000000000BB
:10E5600007E01FF83FFC3C3C781E700E700E700EEA
:10E57000700E700E781E3C3C3FFC1FF807E0000058
:10E58000000000000000000000000000000000008B
:10E590003FE03FF03FF83878383838783FF83FF0C0
:10E5A0003FE03800380038003800380038000000FC
:10E5B000000000000000000000000000000000005B
:10E5C00007E01FF83FFC3C3C781E700E700E700E8A
:10E5D000700E708E79DE3CFC3FFC1FFE07EF0006DC
:10E5E000000000000000000000000000000000002B
:10E5F0003FE03FF03FF83838383838383FF83FF0E0
:10E600003FC038E038F0387038383838381C0000EF
:10E6100000000000000000000000000000000000FA
:10E6200007C01FF03FF0387838383C001F800FF0EB
:10E6300003F00078703878783FF83FF00FC00000A2
:10E6400000000000000000000000000000000000CA
:10E650007FF07FF07FF0070007000700070007004A
:10E660000700070007000700070007000700000079
:10E67000000000000000000000000000000000009A
:10E68000703870387038703870387038703870384A
:10E6900070387038703878783FF03FF00FC0000065
:10E6A000000000000000000000000000000000006A
:10E6B000E038E07870707070707038E038E038E002
:10E6C0001DC01DC01DC00F800F800F8007000000FF
:10E6D000000000000000000000000000000000003A
:10E6E000E187E187718E718E718E718E399C399CB4
:10E6F000399C399C1DB81DB81E781E781E781E786E
:10E700000000000000000000000000000000000009
:10E710007038703838701CE01CE00FC0078007802C
:10E7200007800FC01CE01CE03870703870380000A3
:10E7300000000000000000000000000000000000D9
:10E74000E038E038707038E038E01DC00F800F808E
:10E750000700070007000700070007000700000088
:10E7600000000000000000000000000000000000A9
:10E770007FF07FF07FF000F001E003C007800F0022
:10E780001E003C007800F000FFF0FFF0FFF00000FA
:10E790000000000000000000000000000000000079
:10E7A0003E003E003E003800380038003800380097
:10E7B0003800380038003800380038003800380099
:10E7C0003E003E003E00000000000000000000008F
:10E7D000C000C000600060006000600030003000D9
:10E7E000300038001800180018000C000C00000061
:10E7F0000000000000000000000000000000000019
:10E80000F800F800F8003800380038003800380008
:10E810003800380038003800380038003800380038
:10E82000F800F800F8000000000000000000000000
:10E8300006000F000F001F80198039C039C070E03A
:10E8400000000000000000000000000000000000C8
:10E8500000000000000000000000000000000000B8
:10E8600000000000000000000000000000000000A8
:10E870000000000000000000000000000000000098
:10E880000000FFF0FFF000000000000000000000AA
:10E89000E000600030000000000000000000000008
:10E8A0000000000000000000000000000000000068
:10E8B0000000000000000000000000000000000058
:10E8C00000000000000000001F803FC060E003E087
:10E8D0001FE03CE070E070E071E03FE01E7000007F
:10E8E0000000000000000000000000000000000028
:10E8F000700070007000700077807FE078E07070CA
:10E90000707070707070707078E07FE077800000D9
:10E9100000000000000000000000000000000000F7
:10E9200000000000000000000F003FC039C070E090
:10E9300070007000700070E039C03FC00F00000030
:10E9400000000000000000000000000000000000C7
:10E9500000700070007000700F703FF038F0707041
:10E96000707070707070707038F03FF00F70000051
:10E970000000000000000000000000000000000097
:10E9800000000000000000000F003FC039C070E030
:10E990007FE07FE0700070E039C03FC00F000000F2
:10E9A0000000000000000000000000000000000067
:10E9B00000F001F0038003803FFC3FFC03800380F4
:10E9C00003800380038003800380038003800000B2
:10E9D0000000000000000000000000000000000037
:10E9E00000000000000000000F703FF038F0707071
:10E9F000707070707070707038F03FF01F70007041
:10EA000070F07FE01FC00000000000000000000068
:10EA1000700070007000700073C07FE078F070705C
:10EA200070707070707070707070707070700000C6
:10EA300000000000000000000000000000000000D6
:10EA400003800380000000000380038003800380B4
:10EA50000380038003800380038003800380000021
:10EA600000000000000000000000000000000000A6
:10EA70000380038000000000038003800380038084
:10EA8000038003800380038003800380038003806E
:10EA9000038007000E0000000000000000000000DE
:10EAA000700070007000700070E071C073807F00B3
:10EAB0007F007F007B80718071C070E070E000009B
:10EAC0000000000000000000000000000000000046
:10EAD000038003800380038003800380038003801E
:10EAE0000380038003800380038003800380000091
:10EAF0000000000000000000000000000000000016
:10EB0000000000000000000077CF7FFF71C771C7D1
:10EB100071C771C771C771C771C771C771C700006D
:10EB200000000000000000000000000000000000E5
:10EB3000000000000000000073C07FE078F07070FB
:10EB400070707070707070707070707070700000A5
:10EB500000000000000000000000000000000000B5
:10EB600000000000000000000F803FE038E07070FF
:10EB7000707070707070707038E03FE00F8000004F
:10EB80000000000000000000000000000000000085
:10EB9000000000000000000077807FE078E07070E7
:10EBA000707070707070707078E07FE077807000C7
:10EBB0007000700070000000000000000000000005
:10EBC00000000000000000000F703FF038F070708F
:10EBD000707070707070707038F03FF00F7000706F
:10EBE00000700070007000000000000000000000D5
:10EBF0000000000000000EFC0FFC03C00380038037
:10EC0000038003800380038003800380038000006F
:10EC100000000000000000000000000000000000F4
:10EC200000000000000000001F803FC070E0700086
:10EC30007E003FC007E000E070E03FC01F800000A2
:10EC400000000000000000000000000000000000C4
:10EC500000000380038003800FF00FF00380038027
:10EC60000380038003800380038001F000F0000034
:10EC70000000000000000000000000000000000094
:10EC80000000000000000000707070707070707004
:10EC9000707070707070707078F03FF01F700000CE
:10ECA0000000000000000000000000000000000064
:10ECB00000000000000000007070707038E038E064
:10ECC00038E01DC01DC00F800F8007000700000046
:10ECD0000000000000000000000000000000000034
:10ECE0000000000000000000E38EE38E638C77DC00
:10ECF00076DC36D836D83EF83C781C701C700000A4
:10ED00000000000000000000000000000000000003
:10ED1000000000000000000070E039C039C01F8012
:10ED20000F000F000F001F8039C039C070E00000D5
:10ED300000000000000000000000000000000000D3
:10ED40000000000000000000E0E0E0E071C071C0E1
:10ED500071803B803B801B001F001F000E000E00D7
:10ED60001C007C0078000000000000000000000093
:10ED700000000000000000007FC07FC001C00380D1
:10ED800007000E001C00380070007FC07FC000002C
:10ED9000000000000000000000000100010040022F
:10EDA00023C40FF01FF81FF8DFFB1FF81FF80FF048
:10EDB00023C4400201000100000000000000000028
:10EDC0000000000000000000000000000000000043
:10EDD00030003000300030003000300030003000B3
:10EDE00030003000300030003000300030003000A3
:10EDF0003000300030003000000000800080000152
:10EE000013C209F000F80078187B007800F809F0C8
:10EE100013C200010080008000000000000000001C
:10EE200000000000000000000000000000000000E2
:10EE30000000000000000000000000007C20FFE057
:10EE4000FFE087C00000000000000000000000009C
:10EE5000000000000000000008103030303830386A
:10EE6000303830303078FCFC783000C1814001C04F
:10EE7000804101C0804100C1814001C0804100C18A
:10EE8000814000C1814001C0804101C0804100C17A
:10EE9000814000C1814001C0804100C1814001C06A
:10EEA000804101C0804100C1814001C0804100C15A
:10EEB000814000C1814001C0804100C1814001C04A
:10EEC000804101C0804100C1814000C1814001C03A
:10EED000804101C0804100C1814001C0804100C12A
:10EEE000814000C1814001C0804101C0804100C11A
:10EEF000814000C1814001C0804100C1814001C00A
:10EF0000804101C0804100C1814000C1814001C0F9
:10EF1000804101C0804100C1814001C0804100C1E9
:10EF2000814000C1814001C0804100C1814001C0D9
:10EF3000804101C0804100C1814001C0804100C1C9
:10EF4000814000C1814001C0804101C0804100C1B9
:10EF5000814000C1814001C0804100C1814001C0A9
:10EF6000804101C0804100C1814000C0C101C30394
:10EF700002C2C60607C705C5C404CC0C0DCD0FCF11
:10EF8000CE0E0ACACB0BC90908C8D81819D91BDB81
:10EF9000DA1A1EDEDF1FDD1D1CDC14D4D515D717D1
:10EFA00016D6D21213D311D1D010F03031F133F381
:10EFB000F23236F6F737F53534F43CFCFD3DFF3FD1
:10EFC0003EFEFA3A3BFB39F9F83828E8E929EB2B01
:10EFD0002AEAEE2E2FEF2DEDEC2CE42425E527E791
:10EFE000E62622E2E323E12120E0A06061A163A301
:10EFF000A26266A6A767A56564A46CACAD6DAF6F91
:10F000006EAEAA6A6BAB69A9A86878B8B979BB7B00
:10F010007ABABE7E7FBF7DBDBC7CB47475B577B750
:10F02000B67672B2B373B17170B050909151935380
:10F03000529296565797559594549C5C5D9D5F9F50
:10F040009E5E5A9A9B5B99595898884849894B8B80
:10F050008A4A4E8E8F4F8D4D4C8C44848545874710
:10F060004686824243834181804054532D3120564D
:10F07000455220322E38000004FA97999999D93FC9
:10F08000AF788E1DC571CC3F9FC678D0099AC33F1B
:10F09000935555555555E53F599322942449D23FF0
:10F0A000DE03CB966446C73F44523EDF12F1C23FB7
:10F0B0000000000000000000D8F000080000002060
:10F0C000A00000002871000878F10008A0000020CE
:10F0D000001700004471000800000000000000005C
:10F0E00000000000000001020304010203040607FF
:10F0F00008090204060800000000000000000000EB
:10F1000000000000000000000000000000000000FF
:10F1100000000000000000000000000000000000EF
:10F1200000000000000000000000000000000000DF
:10F1300000000000000000000000000000000000CF
:10F1400000000000000000000000000000000000BF
:10F1500000000000000000000000000000000000AF
:10F160000000000000A24A040000000000000000AF
:08F1700001020304060708096F
:04000005080070ED92
:00000001FF
